:020000040800F2
:1030000000800020F3B600086DB400086FB400081B
:1030100000000000000000000000000000000000B0
:1030200000000000000000000000000071B4000873
:10303000000000000000000073B40008C987000809
:1030400011B3000813B3000815B3000817B3000844
:1030500019B300081BB300081DB300081FB3000814
:1030600021B30008D987000823B3000825B300085E
:10307000C988000827B3000829B300082BB300084B
:103080002DB300082FB3000831B3000833B3000894
:1030900035B3000837B3000839B300083BB3000864
:1030A0003DB300083FB3000841B300084BB7000828
:1030B00043B3000853B7000845B3000847B30008FE
:1030C00001000000000000000A00000000000000F5
:1030D0006400000000000000E803000000000000A1
:1030E0001027000000000000A08601000000000082
:1030F00040420F0000000000809698000000000091
:1031000000E1F5050000000000CA9A3B0000000045
:1031100000E40B540200000000E8764817000000AD
:103120000010A5D4E800000000A0724E18090000AD
:1031300000407A10F35A00000080C6A47E8D030080
:103140000000C16FF286230000008A5D78456301AC
:10315000000064A7B3B6E00D0000E8890423C78A25
:10316000034C206804348047FBE701F0BFFFFEE713
:04317000B0C40008DF
:10317400014802490160704708ED00E00030000892
:10318400B0B51E4D2C1F20688006400F411E032938
:1031940022D81B487944097949008F442301171A1E
:1031A400296803220A40032A00D0164829684906E0
:1031B400490F491C06F0B4FE29684904490E4843E6
:1031C4002968490F491C06F0ABFE0BE07D20000284
:1031D40008E00120C00305E00C3D28688004410F8D
:1031E4000848C84008490860226892093C231340F3
:1031F400064AD258D0400860B0BDC0460C10024008
:1032040000127A000024F4005C0B00205CB100087A
:1032140010B5816A8B6D8A6D5024234205D0D20685
:1032240002D4096D496B884710BD012043021A433B
:103234008A650A68D3681B059B0F02D0104908678A
:1032440010BD8B7E002BF9D113681B07F6D593684C
:103254005B0709D4583153680C24A3435360FF23FC
:1032640002330A689A4305E08A6D202313438B6571
:10327400CA6D5C3102430A600149086710BDC0464B
:04328400E809002035
:10328800F0B587B005460020049006900124E602B8
:10329800E94A1068E949884206D03246AC32E84823
:1032A800E84906F095FFE44A2868E74988420DDCBA
:1032B800F449884218DDF44988422ADCF6498842F4
:1032C80042D0F64988423FD0F5493BE0DF49884281
:1032D80014DDDF49884224DCE149884234D0E149E1
:1032E800884231D0E0492DE0EE49884221DDEE499F
:1032F800884229D0012827D0EC4923E0DB498842BD
:103308001CDDDB4988421FD0DA4988421CD0DA49E3
:1033180018E0DE49884217D0DD49884214D0DD49DB
:1033280010E0CC4988420FD0CB4988420CD0CB4919
:1033380008E0DF49884207D0DE4903E0CF498842E8
:1033480002D0CF49884269D10595A868002809D0DC
:10335800D949884206D03246AE32B948B94906F052
:1033680037FFB54A3546106904263043D34FB84273
:1033780007D105984068401E02281AD32A46B3325E
:1033880012E0D069401E082806D32A46B732AC4856
:10339800AC4906F01DFFA84A059840680221C841BB
:1033A800082806D32A46B932A548A64906F010FFD0
:1033B800A14A5423D05C012802D1022007B0F0BDF5
:1033C800D45410688168490717D41169059A52685E
:1033D800022A17D104221143B9422BD1B849C94353
:1033E800059A1268D3430B43816A194054238162BA
:1033F8000024002A23D4904AAAE0906D202101439A
:103408009165A5E003933143B942AD4F24D1059CA2
:1034180021680F40826A3A4382628BE03246AD32BD
:103428008748884906F0D4FE834A0595A86800288D
:103438008ED197E7059802680024002ADBD5A248B8
:103448000168994B9A424FD09A4B9A424FD0984B69
:103458009A4255D1052248E01F2313400F240194B6
:103468009C407549096EA143029105990968394242
:1034780037D0CF07049F4BD18F0744D44F0744D48C
:103488000F0744D4CF06374642D48E0600D5BAE09B
:103498004E0600D5B9E00E0600D5B8E0CE0500D539
:1034A800B7E08E0500D5B6E04E0500D5B5E0294257
:1034B80000D0B4E0CE0400D5B3E08E0400D5B2E06D
:1034C8004E0400D5B1E00E04019F21D4CE0300D5EF
:1034D800ADE08E0300D5ACE04E03F6171227374057
:1034E80016E04E00F70E13E00322920501E00322D6
:1034F800D2051140072292050368934359180160C9
:103508004D4A542324E0012702E0022700E0032764
:103518009F40029D2F43484E37669208F6699642AF
:1035280007D9E243846A14408A00120F9A40224362
:103538008262059C0A0243699343A4681440614A65
:1035480022401A4342610024002906D43A4A039BC8
:103558000498D054204607B0F0BD01265A480068A8
:103568000722930502461A40514FB94230D1F70558
:1035780005463D402CD154490868984302433A43D4
:103588000A6052480068524906F0C8FC0C214143C1
:10359800481C069006980028D8D0274A039B06980E
:1035A800401E069006980028D2D00698401E069025
:1035B80006980028CCD00698401E06900698002849
:1035C800C6D00698401E069006980028E7D1BFE7A7
:1035D800354DA9420AD1370605463D4006D13A493C
:1035E8000868984302433A430A60AFE7314DA9425D
:1035F800ACD1B1050840A9D1334D2868984302439E
:103608000A432A60A2E7052782E7062780E70727FB
:103618007EE708277CE709277AE70A2778E70B2758
:1036280076E70C2774E70D2772E70E2770E7102757
:103638006EE711276CE7C046640A002000240140A9
:10364800EDBF000890BD0008FF000020FF1F0034F8
:10365800FFFF004000000140000002440000044851
:1036680000200034004000380080003CFF030028A0
:10367800000400280008002C001000300001002081
:1036880000020024030000081F000014200000149A
:10369800400000188000001C040000080800000C0E
:1036A80010000010FF3F00B8004000B802000004FE
:1036B800001000B0002000B404FFFF0704000080E1
:1036C800FFFF070000FFFF07082701405C0B0020F1
:0436D800400D03009E
:1036DC00F0B58DB00446002306930120002C00D1D8
:1036EC00D2E121680A68002A00D5CDE103930427B2
:1036FC003943FF250235404EB14203D120690028E1
:10370C0008D113E03D483E492A4606F05FFD20698A
:10371C0000280BD001210A02904207D049028842AE
:10372C0004D06A1C3548364906F050FD6069F841F2
:10373C00092804D3AA1CD648D64906F047FD012710
:10374C00F803E1690143814204D0EA1CD048D14915
:10375C0006F03CFDB904E06808430191884204D0AE
:10376C002A1DCB48CB4906F031FDA0691021C84178
:10377C00042804D36A1DC648C64906F027FD206AF2
:10378C00C549884208DC002814D03905884211D07C
:10379C00790588420ED008E0B90588420AD0F905AF
:1037AC00884207D03906884204D0AA1DB848B949C6
:1037BC0006F00CFD606A322800D96DE0784400797F
:1037CC00400087441F696969696969696969696940
:1037DC0069696969691F1F696969696969696969E1
:1037EC0069696969691F1F696969696969696969D1
:1037FC0069696969691F1F0004020140EDBF000877
:10380C0016BA0008606800280DD0F90288420AD068
:10381C000321C902884206D02A4608329C489D4999
:10382C0006F0D4FC606822462832002812D0A0682A
:10383C0002280FD3B90388420CD005210903884212
:10384C0008D00B359248934916462A4606F0BEFC22
:10385C0032468E4E0492507800284FD10025E562F6
:10386C0015700C950B950A95099508950520000780
:10387C002168B14219D0894A91423FD188490A68DE
:10388C003A430A6009683940079102210891079967
:10389C00F902059102901EE0EA1D7D487D4906F073
:1038AC0095FC60680028B0D1BDE77D490A683A43B1
:1038BC000A600A683A400792079A0A6802231A4378
:1038CC000A600968194007910C21089107997549FC
:1038DC000291202105910A950321099108AE3146E8
:1038EC0000F0E6FA07200C900B950A95022009903F
:1038FC00059808900298314600F0DAFA0597256889
:10390C00286802902A686849114026460C364CCE2D
:10391C001E43A369E769206A3043184338431043B8
:10392C000843286061680320C00281425B4E09D0C5
:10393C000598C20291420DD1306890433060716895
:10394C0011430DE00598C002316801433160716884
:10395C00814305E03068554A104030607168114071
:10396C00039F7160A16801290DD0052000038142DD
:10397C000ED005988203914212D13068104330600A
:10398C007168914312E0059880033168014303E0AC
:10399C00059880033168814331607168014305E00B
:1039AC003068434A1040306071681140716028687B
:1039BC008006800F26D030200299014022D13D484C
:1039CC0000683D4906F0A8FA142141430691069877
:1039DC00002817D00698401E06900698002811D093
:1039EC000698401E0690069800280BD00698401E9C
:1039FC0006900698002805D00698401E069006985A
:103A0C000028E7D1B5420FD0019D616A8A072B4887
:103A1C0010D0CB062A4B11D41C68AC431C608C060E
:103A2C0011D55C682C4310E005984504616A8A073F
:103A3C002248EED10168A943016019E01C682C43AF
:103A4C001C608C06EDD45C68AC435C60DD601D6171
:103A5C00002A08D40268AA430260C90708D0011FD3
:103A6C000968294307E002682A430260C907F6D1B6
:103A7C00011F0968A943049A001F016050780028AF
:103A8C0001D10598507038460DB0F0BD04020140CC
:103A9C00EDBF000816BA0008FFFF3F00000201400E
:103AAC0034100240000400500F7400FEFFF7FFFFBB
:103ABC00FFBFFFFF5C0B0020400D03008418024089
:043ACC00001802409C
:103AD00070B582B00026019600280DD0054600681A
:103AE0000168002908D4042108432149884206D1ED
:103AF0002920285C01280BD0012002B070BD1D4890
:103B00001D491E4A06F068FB2920285C0128F3D1D4
:103B100028682935016801220A43026002202870C2
:103B200017480068174906F0FDF9C0000190019898
:103B300000281AD00198401E01900198002811D049
:103B40000198401E0190019800280BD00198401E5A
:103B500001900198002805D00198401E019001981D
:103B60000028E7D1304602B070BD02B070BDC0463B
:103B700004020140EDBF000816BA00081F03000050
:083B80005C0B0020400D030066
:103B8800F0B585B0574C2178002902D0022005B045
:103B9800F0BD02900393012727707D20C100606A61
:103BA800049141183E04504D2868304216D0636A8B
:103BB80003208B421AD22B6833420FD0636A8B42A0
:103BC80014D22B68334209D0636A8B420ED22B6819
:103BD800334203D0636A8B42E6D307E0286843493F
:103BE8004B1C01932B600842384603D000212170FA
:103BF80005B0F0BD606A049941180120009087045F
:103C08002868384216D0636A03208B42EED22B68AC
:103C18003B420FD0636A8B42E8D22B683B4209D003
:103C2800636A8B42E2D22B683B4203D0636A8B42C1
:103C3800E6D3DBE7686800990843686002990A6080
:103C4800BFF36F8F03984860606A04994118286829
:103C5800304216D0626A03208A4219D22A68324258
:103C68000FD0626A8A4213D22A68324209D0626A45
:103C78008A420DD22A68324203D0626A8A42E6D367
:103C880006E028680199296018490842009807D079
:103C98006968009A914369600021217005B0F0BD00
:103CA800606A049941182A6800203A42F0D0636A91
:103CB80003228B4213D22B683B42E9D0636A8B42C2
:103CC8000DD22B683B42E3D0636A8B4207D22B6844
:103CD8003B42DDD0606A88421046E4D3D8E703202F
:103CE800D6E7C046E809002010200240FAC30000C9
:103CF800F0B587B00446684D287C002804D1674891
:103D08006749A02206F064FA2878002802D0022029
:103D180007B0F0BD0594012129707D20C200686AB2
:103D2800069282180C045F4E3068204219D06B6AE4
:103D38000320934211D23368234212D06B6A934214
:103D48000BD2336823420CD06B6A934205D2336896
:103D5800234206D06B6A9342E6D30021297007B04C
:103D6800F0BD3068504B5A1C049232601842084625
:103D7800F3D1686A069941180120039087043068D6
:103D8800384216D06A6A03208A42E6D232683A423A
:103D98000FD06A6A8A42E0D232683A4209D06A6A27
:103DA8008A42DAD232683A4203D06A6A8A42E6D351
:103DB800D3E70022D04305990860287DA96C08182C
:103DC80081425AD201924029029106D3334834499C
:103DD800364A06F0FDF90299334B7068344A1040B0
:103DE800C9000143A01C08437060686A069941181D
:103DF8003068204216D06A6A03208A4240D232686C
:103E080022420FD06A6A8A423AD23268224209D0E4
:103E18006A6A8A4234D23268224203D06A6A8A4283
:103E2800E6D32DE0306804993160184227D1686ADA
:103E3800069941183068384216D06A6A03208A42C7
:103E48001ED232683A420FD06A6A8A4218D2326861
:103E58003A4209D06A6A8A4212D232683A4203D098
:103E68006A6A8A42E6D30BE0287DA96C0818029991
:103E7800491C8142A7D3019805E0002003E003987C
:103E88000599029A0A6071680222914371600021C3
:103E9800297007B0F0BDC046E8090020EDBF000852
:103EA80080BA000810200240FAC300005202000045
:043EB80005FEFEFF06
:103EBC00F0B58DB00B4604460B20000721180A20E4
:103ECC00C141039104290C9307D3052905D09848C7
:103EDC009849B12206F07AF90C9B1868010C02D1B2
:103EEC0080B2002805D192489249B22206F06EF9B0
:103EFC000C9B58689049884207941CDC122800D906
:103F0C000BE1012181408D48014200D105E1986807
:103F1C00032805D386488749B42206F057F90C9B31
:103F2C001A68002A00D1EAE0012005908B488442EF
:103F3C000FD005200EE08249884200DDE1E0844983
:103F4C008842E4D083498842E1D083498842DED05C
:103F5C00E3E003200190059D2804029000270B97B5
:103F6C003C46099711E021437160089C1A68104681
:103F7C00E840BF1C0B99091D0B9108346D1C099965
:103F8C00491C0991002800D1B9E0681E059E0A90D1
:103F9C0086403240EAD0586812280492089423D8FC
:103FAC0001218140704A11421ED0D868042806D3E2
:103FBC00C4225F485F4906F009F90C9BD868B840E9
:103FCC000321B940079CA2688A430243A260586847
:103FDC00C206D20F0A9B9A406368B34313436360D3
:103FEC000C9BCA433E4605E00321B940CA430999DC
:103FFC004E00079CE168069211409A68B2400A4351
:10400C00E2601021014312291DD10398042841D2EA
:10401C001869082806D3DD224548464906F0D6F82B
:10402C000C9800691C210B9A11400F228A400A9BA4
:10403C00DB089B00E3181C6A944388402043079CD0
:10404C0018620C984068226806990A4003210346BE
:10405C000B40B340134323600C9BC000089C85D5D8
:10406C00182020400F2383400A9A8A433C4EB118F3
:10407C000A6E9A43603105231B07079C9C4212D0A1
:10408C003A4B9C4211D03A4B9C42019B049C0ED162
:10409C0002230CE00528BBD0DC222548254906F07C
:1040AC0095F80C9BB4E7002300E00123049C8340AB
:1040BC0013430B602B4801680C9B5868029A104202
:1040CC0001D0214300E0A143264A116051688203CC
:1040DC0001D5214300E0A143224A51603168C2025C
:1040EC0005D5214331607168800206D53BE7A143B9
:1040FC0031607168800200D535E7A14334E70DB01B
:10410C00F0BD1049884200D101E70F49884200D127
:10411C00FDE60E49884200D1F9E605480549B3226F
:10412C0006F054F80C9B9868032800D3F2E6F7E6E7
:10413C00EDBF0008EEBA0008FFFF10100F000600DC
:10414C00FFFF21100000221000003110000032107F
:10415C00000011100000121000002110000C005083
:10416C0000180240801802400600060000040050AF
:04417C0000080050E7
:10418000F0B581B00446744B00280CD0201F0221EA
:10419000C84103280CD88000704908581946042CDF
:1041A0000BD175310AE01946743118466E3005E0BE
:1041B000184673301946042CF3D077310778186B02
:1041C0000D780126B107009188420BD064498842DE
:1041D00008D0644988420BD102212246CA41062AEE
:1041E0000FD21EE002212246CA41042A09D218E059
:1041F000002C02D15C49884213D05C49884200D12E
:10420000A4E05B494118B002814348424841002C78
:1042100001D1002805D157485749584A05F0DCFF1D
:104220004D4B012F00D083E0012D00D080E0002C09
:104230000FD0211F0220C14103291DD879440979DB
:1042400049008F44011E23296F215854042C21D189
:1042500026E06E2002211954742019541D6B484A1F
:10426000954223DC0098854238D03D48854235D0C0
:104270003D48854232D029E073215854042C09D19D
:104280000EE070215854042C04D109E071215854D7
:10429000042C05D0772104E072215854042CF9D164
:1042A000752158541D6B364A9542DBDD35488542F1
:1042B00006DC2C48854211D02C4885420ED005E002
:1042C000314885420AD03148854207D029482A49D9
:1042D0002F4A1F4605F080FF294A3B46022120460F
:1042E000C841062826D21F2004403046A040296A33
:1042F00081432962296A01432962186B904206DCD6
:104300000099884209D01649884206D00DE0174925
:10431000884202D01349884207D182681D49114062
:10432000062905D03204914202D001683143016070
:1043300001B0F0BD0F28D6D01548421C0D480E49DB
:104340001F4605F049FF0E4A3B46CCE704212143B6
:10435000042900D165E754E76C0900200CB200087D
:1043600000040040002C01400020004000400140BB
:1043700000BCFEBFEDBF0008CBBE00082408000053
:10438000FF2B0140FF430140004401400048014031
:08439000F41D0000070001000C
:10439800F0B583B00E4604468548006B854D8649C6
:1043A800884209DD8549884211DC8749884219D04D
:1043B8008649884216D010E001218907884211D029
:1043C800834988420ED0834988420BD005E07C4956
:1043D800884207D07B49884204D07F487F492A46D3
:1043E80005F0F6FE20680A2840D8012181407C4863
:1043F80001423BD06068401E032804D3AA1C7648BB
:10440800764905F0E5FEA0680227F841042804D3A0
:10441800EA1C7148714905F0DBFEE068102804D3F6
:104428002A1D6D486D4905F0D3FE6C226049885CF1
:10443800012800D1B9E001278F54042E02921FD021
:10444800002E28D1096B086AB84308625A4881428D
:104458008D69E0680190226860680B6A4FDCBE07CE
:10446800B14252D05A4EB1424FD083E06A1C5A48EA
:104478005A4905F0ADFE6068401E0328BED2C2E767
:10448800086B4D49884244DCB90788424FD05049EF
:1044980088424CD043E0086BB90788420DD04C499C
:1044A80088420AD04849884207D03A354A484B4999
:1044B8002A4605F08DFE3E48006B3903026A8A439E
:1044C800026261680902474A0A40E168090389B241
:1044D8008918F3221202C36993430B43016AC3612B
:1044E8000522520323681B0313409143C918016234
:1044F80003218902C2698A43C2611C3037E0334E06
:10450800B14202D0304EB14234D10326B5430543FF
:1045180031E02D4988420AD02C49884207D01A3503
:104528002D482E492A4605F053FE2148006B016AA2
:10453800102291430162616809022A4A0A40E1682F
:10454800090389B28918F3221202836993430B4342
:10455800016A836122681201A0231A4099438918CD
:1045680001620321890282698A4382611830A16845
:10457800090213E03D4308461830F026B543019E72
:104588003601F6B2AD198D610A252A40AB439A1857
:104598000A628A690C239A438A61A1680027044A3F
:1045A800029BD75402680A430260384603B0F0BD44
:1045B8006C090020EA0F0000FF2B0140FF43014077
:1045C8000044014000480140002C014000400140E7
:1045D8000004004000200040EDBF0008CBBE0008EA
:0845E80005040000000FFFFFB5
:1045F000F0B583B09748401C974F79688142974E39
:1046000004D397489749324605F0E6FDB86800287C
:104610000BD001210A03904207D00907884204D039
:10462000721C8F488F4905F0D7FDF86839688E4CA9
:10463000A14212D00C21C841042805D332460832C9
:104640008748884905F0C8FD0120C002396A014346
:1046500081420CD03246093205E00121490308436A
:10466000884204D0321D7E487E4905F0B5FD386988
:1046700000280DD001218902884209D00321490276
:10468000884205D032460C327548764905F0A4FDC3
:1046900078690C25002801D0A84305D032460D3298
:1046A0006F48704905F098FD0195B8690821C84127
:1046B000042805D332460E3269486A4905F08CFD5C
:1046C00001200290C503F8692843A8424FD1786AB7
:1046D0000C2805D31036F048F049324605F07CFD31
:1046E0003E683168EF480840B9683A690A437B6917
:1046F0001343F9690B437A6E1A4302433260032075
:104700000090000372688243F868104370600022D2
:10471000A642104600D0386ABB690343B068E24C39
:1047200004401C43B460F06A0F2398433C467B6A04
:104730001843F062DD4886420DDDDD488642D84FE1
:1047400026D0BE421DD0DB4886420BD1DC48C06C6F
:104750008007000F1AE0D84886425FD0D7488642CB
:10476000CF4F15D01022D848BE4214D160E0324657
:104770000F32C948C94905F02FFD786A0C28A9D223
:10478000AEE7CF48C06C000A019A1040CD4A1258DB
:10479000CD48BE424CD0A94220D1082A00D974E0AD
:1047A000274652007A4492885200974408006301D9
:1047B000360163017C006301630163018800C34823
:1047C0000068BF490968890A1C220A40C049895803
:1047D0001F220A40D04000D01FE14AE1082A54D8E5
:1047E000274652007A4492885200974408004301B9
:1047F000330143016A004301430143017600B3489A
:104800000068AF490968890A1C220A40B0498958E2
:104810001F220A40D04000D01CE12AE1A848C06C09
:10482000019A1040A74A12589D4FA748BE42B2D1E4
:10483000082A2AD8274652007A4492885200974480
:1048400015001901C60019012600190119011901E5
:10485000C400C04600127A00DC080020150C0000DD
:10486000EDBF000858BB0008008000409748006872
:1048700093490968890A1C220A40954989581F22D0
:104880000A40D04000D0A2E0F3E02746F2E08C4C92
:1048900021688906490F22D0226838210A40082A57
:1048A00023D17C4893E0864C21688906490F3CD08F
:1048B000226838210A40082A43D17648ADE02846CC
:1048C000ABE07F4C21688906490F34D0226838213B
:1048D0000A40082A55D16F48BCE02846BAE0083C97
:1048E00021688904490FC84071E022680A40102AF3
:1048F00067D11D466168009A11400329654A00D0BE
:10490000024660684006400F411C104605F00AFB55
:1049100061684904490E48436168490F491C05F024
:1049200001FB2B46002852D1A3E0083C21688904F2
:10493000490FC84071E0083C21688904490FC8400C
:1049400088E022680A40102A5CD11D466168009AFE
:10495000114003294F4A00D0024660684006400FCC
:10496000411C104605F0DEFA61684904490E4843CF
:104970006168490F491C05F0D5FA2B4600284CD137
:1049800077E022680A40102A59D11D466168009AD2
:10499000114003293F4A00D0024660684006400F9C
:1049A000411C104605F0BEFA61684904490E4843AF
:1049B0006168490F491C05F0B5FA2B46002849D11A
:1049C00057E02068084020285CD10120C00359002E
:1049D000404A515A05F0A6FA7A6800995143884234
:1049E00048D31103884245D8010E54080002002321
:1049F0000019594105F0BAFA38494118384A91422C
:104A000035D337E0206808402028284605D02068A4
:104A1000084018282CD17D20000259002D4A515AF7
:104A200005F080FA400079684A08101805F07AFA13
:104A3000294901401ED00007400F084317E02068B5
:104A400008402028284605D02068084018280FD1A3
:104A50007D20000259001F4A515A05F063FA796817
:104A60004A08101805F05EFA80B2102802D3F060F0
:104A7000002002900020386778671A48B8660298CC
:104A800003B0F0BD206808401828F1D17D20000255
:104A90009DE7C04600127A00EDBF000858BB000831
:104AA00000800040F369FFCFFFF4FF11FF4B00408F
:104AB000004C0040003801400044004000480040E5
:104AC00008100240BCB100080024F4005C0B002078
:104AD0009CB100088EB80008F0FF000000FDFFFF49
:084AE00000FD0F0001000100C0
:104AE80070B5774DA86A010A764C0FD1C10715D168
:104AF800810728D441073CD4010750D4C10664D4A7
:104B0800810678D4400600D58BE0C0E06E486F4936
:104B1800224605F05DFBA86AC107E9D001214E04D1
:104B2800E96A0A463243B24206D0621D66486749BE
:104B380005F04EFBA86AE96A2A685368B3430B4339
:104B480053608107D6D501210E04296B0A463243EA
:104B5800B24207D022460C325B485C4905F038FB6C
:104B6800A86A296B2A685368B3430B43536041070B
:104B7800C2D501218E04696B0A463243B24207D07E
:104B8800224613325048514905F022FBA86A696B46
:104B98002A685368B3430B4353600107AED501211C
:104BA800CE03A96B0A463243B24207D022461A32D4
:104BB8004548464905F00CFBA86AA96B2A68536862
:104BC800B3430B435360C1069AD501210E03E96B29
:104BD8000A463243B24207D0224621323A483B497C
:104BE80005F0F6FAA86AE96B2A689368B3430B43A1
:104BF8009360810686D501214E03296C0A4632430B
:104C0800B24207D0224628322F48304905F0E0FA50
:104C1800A86A296C2A689368B3430B4393604006DB
:104C280035D528682A49884208D02A49884205D0BB
:104C380022462F322448254905F0CAFA01200605E4
:104C4800696C08463043B04206D0224630321E48CE
:104C58001E4905F0BDFA696C28684268B2430A43E8
:104C68004260B14213D1A96C15220B46D341042BE3
:104C780007D3224635321448144905F0A9FAA96C1D
:104C8800286803225205436893430B434360282056
:104C9800285C000612D50120C604E86C01463143A1
:104CA800B14206D03D3408480849224605F090FA3A
:104CB800E86C29684A68B24302434A6070BDC0463E
:104CC800DC080020E10C0000EDBF000858BB00081C
:084CD8000044004000380140D7
:104CE000F0B581B08C20364900220A50354B5C6A01
:104CF00008680168090716D5C169890213D4012122
:104D00004F050091CE02304D02E0C16939420AD10F
:104D1000596A091BA94201683DD84907F5D5C169FF
:104D20003142F2D018E00168490728D5C16949022B
:104D300025D401218F050091CE02234D02E0C169E7
:104D400039421CD1596A091BA942016823D8490775
:104D5000F5D5C1693142F2D006620D2149010368DF
:104D60008B4303608168009B9943816084202021EC
:104D7000134C215020468C302346883318E0842081
:104D800020210F4C215088202150E26610468021BE
:104D9000625401B0F0BD0D235B019943016081684D
:104DA000009B99438160064C20468830234684331B
:104DB00020211960016003208021625401B0F0BD00
:0C4DC000DC080020E8090020FFFFFF01D4
:104DCC0070B58421415821291AD102465632938A52
:104DDC00002B15D00168104C02E05B1E1D040FD097
:104DEC001588002D0DD0CD692D06F6D5056D2E88B4
:104DFC0026408E62AD1C056515886D1E1580ECE78E
:104E0C0070BD0120C0058A6882438A600868402210
:0C4E1C0002430A6070BDC046FF010000A8
:104E280010B58421415821290FD1014656310A88ED
:104E3800002A0BD0026D1388094C1C4003689C6241
:104E4800921C02650888401E088010BD0068016831
:104E5800802291430160016840220A43026010BD2C
:044E6800FF01000046
:104E6C00F0B586B00168CA690F688E688823C3588C
:104E7C00222B79D105465E3520246B89002B0094BA
:104E8C0075D0224073D03246064688366B88039321
:104E9C0001231A40049205931A0217400197876D5B
:104EAC00029502E0C266A20661D5496A039A1140D6
:104EBC0039702988491E2980816D4F1C87650168CE
:104ECC00CC6962072AD0019B5D425D41E307059BDB
:104EDC0000D02B46002B04D101230B6275681D43B7
:104EEC007560049B5D425D41A307059B00D52B4675
:104EFC00002B05D102230B62736804251D437560DA
:104F0C00049B5D425D41002A059A20D4002A20D0E2
:104F1C007268002A029D01D0002272602A88002A41
:104F2C00C1D1012212020B6893430B608A68194BA2
:104F3C001A408A602022326000220267C36E012B65
:104F4C00B0D10B681025AB43029D0B60AAE72A0079
:104F5C00DED104220A627268022313437360726802
:104F6C00002A029DD8D1D9E7183108220DE02A88F1
:104F7C00002A0DD06B899A420AD2074A026705486B
:104F8C00401C8A6802408A60009A086810430860D6
:0C4F9C0006B0F0BDFEFFFFEF9DB3000863
:104FA800F0B586B004460168CA690B688D68882028
:104FB800205822287BD10495019325465E35202070
:104FC80000906889002875D00098024072D0264663
:104FD800883668880390012204981040049005924E
:104FE80010021A4602400192A76D029402E0E2669E
:104FF80098065FD5486A039A104038802888401E72
:105008002880BF1CA765CB695A072AD0019844425B
:105018004441D807059800D02046002804D1012033
:1050280008627468044374600498444244419807D1
:10503800059800D52046002805D10220086270682E
:10504800042404437460049844424441002A0598A7
:1050580020D4002820D070680028029C01D00020AD
:10506800706028880028C3D1012000020A688243A2
:105078000A608868194A1040886020203060002241
:105088002267E06E0128B2D108681024A043029C70
:105098000860ACE72000DED10420086270680222B4
:1050A8000243726070680028029CD8D1D9E7183191
:1050B80008220DE0288800280DD06A8990420AD27B
:1050C800074820670548401C8A6802408A60009AA1
:1050D80008681043086006B0F0BDC046FEFFFFEF49
:0450E80007B4000801
:1050EC0000B5C7B0AD4A1068FF21359160313791DA
:1050FC005F393291084310607D203890C400A84E6F
:10510C003068214604F008FF401E010E01270029DB
:10511C0028D1A4494860A44A1368A44E3340032004
:10512C0085075B19136000238B6007230B601168E4
:10513C0031409B4E11609E490F719E4BD96839438B
:10514C00D960D96839404291429939079A680A4323
:10515C009A609A680A4042924299400296490A68BB
:10516C0002430A6003203A904202944D28461438B8
:10517C0001683092914301223B9252023492891879
:10518C00016031682868319426461836304229D09F
:10519C00062048438A4904F0BFFE0221081A03285E
:1051AC0020D0821E514251412A6832423A4600D0E8
:1051BC000A46002A16D1421E514251412A683242F7
:1051CC003A4600D00A46002A0CD1414241412A6895
:1051DC0032423A4600D00A46002A03D1001D296803
:1051EC003142DCD13397734C27462C3F3968254626
:1051FC00283D28683A9A8243382039900140102380
:10520C000846369358408018434243413B98420429
:10521C00204634380829016825D0002B23D13B9B2C
:10522C001B041943016062494B6A046814421AD189
:10523C004C6AE41A642C14D80468144213D14C6AD6
:10524C00E41A642C0DD8046814420CD14C6AE41A8C
:10525C00642C06D80468144205D14C6AE41A652CF7
:10526C00E3D372B6FEE72E964C49096807212F91BD
:10527C0009033B680B433B603B68524C23403B604B
:10528C0003681342399C01D172B6FEE73A683B9B26
:10529C001A4306232D939A433A60454A526A3B6857
:1052AC002340082B21D0424B5B6A9B1A464EB342DB
:1052BC00EAD83B682340082B17D03D4B5B6A9B1AFE
:1052CC00B342E1D83B682340082B0ED0384B5B6AC5
:1052DC009B1AB342D8D83B682340082B05D0344BDB
:1052EC005B6A9B1AB342DAD9CEE72C4A1268520792
:1052FC002CD02A4E32682F9B9A4332602C4A526A29
:10530C00264B1B685B0721D0294B5B6A9B1A2E4EE0
:10531C00B342B9D8214B1B685B0717D0244B5B6A8F
:10532C009B1AB342B0D81D4B1B685B070ED0204BA9
:10533C005B6A9B1AB342A7D8184B1B685B0705D056
:10534C001B4B5B6A9B1AB342DAD99DE73A688A43D6
:10535C003A6039688906490F3CD0386820400828E3
:10536C001A483CD039682140102900D03FE1296807
:10537C003A9A11400329389C00D0154829684906EF
:10538C00490F491C04F0C8FD29684904490E4843DB
:10539C002968490F491C04F0BFFD21E000200240A0
:1053AC005C0B002010E000E020ED00E0FFFFFF00B0
:1053BC00E809002034100240000001401470004045
:1053CC0040420F00FFF0FFFF8813000000127A002C
:1053DC000024F40000688004410FCB48C840389C7E
:1053EC00396889093C252940C84A51581F2739403A
:1053FC00C840C7490860E10004F08EFD401EC54955
:10540C00884200D940E7C4490979C44A5060C44C69
:10541C002068C04B18403A9B9B07C01820600026A0
:10542C0096602F981060002900D12DE720972068F6
:10543C00B849084020603398B74908712B95B94C8E
:10544C00206A3A9A90432062206A23939843206200
:10545C003B9DA805216A81432162469645962068AA
:10546C0004212C9108432060206808403D903D9811
:10547C0020682021389108432060206808403D9026
:10548C003D98206828432060206828403D903D9836
:10549C0020680221084320602068259108403D9037
:1054AC003D98206808212A91084320602068084014
:1054BC003D903D989C480F2129910161449643925F
:1054CC0014469A4842909A481838289042AF394668
:1054DC00FEF7EEFC449643942C984290954839463E
:1054EC00FEF7E6FC44964394E8031C90401C429063
:1054FC0005201F90000721903946FEF7D9FC4496F1
:10550C00439428041E90223842908B4C20463946F6
:10551C00FEF7CEFC449543962A9842902046394695
:10552C00FEF7C6FC459644964395299842907E48D2
:10553C0018383946FEF7BCFC40207D49086144967A
:10554C0043951D90429028983946FEF7B1FC754959
:10555C0048682843486048682840429042983598EB
:10556C000002764A116881431160754934980860CD
:10557C00744A2B9815542C20289015546F070C2026
:10558C002290106456649664D76416632F98506307
:10559C00906356629662101D06772C98D0619576B2
:1055AC00168369052C056848199051C2166027911D
:1055BC0051602A9890603F963E963D9626960C3AFE
:1055CC003C96D068389908432028379D06D02A4647
:1055DC0036325E485E4904F0F9FD5A4A10690028DB
:1055EC000CD50121C907884214D05A4909E0386802
:1055FC00204020283BD13B98C003F0E60AD03B99D1
:10560C004905884206D02A4637325048504904F0A2
:10561C00DDFD4C4A907E022806D32A4638324B4890
:10562C004B4904F0D3FD474A906A0A211B91C841AB
:10563C00042806D32A4639324448454904F0C6FDAD
:10564C00404A506A4449884207DC4449884215DC88
:10565C00002823D0012189021DE04149884214DC35
:10566C0013218901884219D01F99090213E0386867
:10567C002040182800D181E10020B0E611218901D9
:10568C0088420BD00921C90105E015218901884206
:10569C0004D017218901884200D072E12898105C4F
:1056AC00022806D32A463B322848294904F08EFDAD
:1056BC00244A5069042808D0082806D02A463C32CF
:1056CC002248234904F082FD1E4A3B980103106BCB
:1056DC0008431A91884245D1107E02284CD2507E44
:1056EC00022853D2506B08285AD2906B082861D2EA
:1056FC002B98105C022868D2D06C3843B8426FD11A
:10570C001069002876D18FE00024F4005CB1000809
:10571C005C0B0020FFFFFF00E809002010E000E018
:10572C0020ED00E034100240180C0050C0E00000E6
:10573C0018080050001400500004005008E400E069
:10574C0000E100E0640A002000240140EDBF0008E5
:10575C0090BD000804000080BF0400003F0400005E
:10576C003F0500002A463D32FB48FC4904F02EFD63
:10577C00FB4A107E0228B2D32A463E32F648F7493D
:10578C0004F024FDF64A507E0228ABD32A463F3261
:10579C00F148F24904F01AFDF14A506B0828A4D3E1
:1057AC002A464032EC48ED4904F010FDEC4A906B6F
:1057BC0008289DD32A464132E748E84904F006FD03
:1057CC00E74A2B98105C022896D32A464232E248CC
:1057DC00E24904F0FBFCE24AD06C3843B8428FD06B
:1057EC002A464432DC48DD4904F0F0FCDC4A1069FE
:1057FC00002819D03899515C022907D32A4648321F
:10580C00D548D64904F0E2FCD54A1069279988425C
:10581C000AD1D069401E082806D32A464C32CE48FD
:10582C00CE4904F0D3FCCE4A3898105C012809D13B
:10583C00907E012806D12A465232C748C74904F047
:10584C00C5FCC74A906D002800D0D7E024970027EC
:10585C00469745971068C349884200D0CAE0C249B0
:10586C00C8682043C860C8682040419041980868C7
:10587C000125284308600868284041904198086831
:10588C00022210430860086817921040419041981A
:10589C00449703264396E020429042AC219821463F
:1058AC00FEF706FB44971596439618954295AF481C
:1058BC002146FEF7FDFAAE4E376280200521AD4A37
:1058CC00121D32607160B760F7603061329971619E
:1058DC002E99B1613899F161306A2299C841042836
:1058EC0004D39D48A449A82204F070FC70683E289B
:1058FC0004D39948A049AA2204F068FC25211798E2
:10590C00169170549D481030356829680140296003
:10591C009B488030B0649B482818142104F0FCFA92
:10592C00800097494118306417917164E8B20838C7
:10593C00142104F0F1FA20990840189C214681406A
:10594C00F164B068F26802433369134372691A4315
:10595C00B3691343F2691A43336A13432A681A432F
:10596C002A602546A203904218D10020179A106095
:10597C007060854A11600346014628E0389C20027D
:10598C002EE52A463A327448744904F01FFC744AD6
:10599C002898105C022800D384E68AE67068C4B2AA
:1059AC00179A1460784A1160401E032838463B460B
:1059BC0039460CD8611E88001018C367159B0B4024
:1059CC0029469940714B19607C30BC321346F76301
:1059DC00169AB5542422B75430657365B165604A84
:1059EC001665B2626A4B586835998843586028032B
:1059FC006849086054201754D765249F3B980507C5
:105A0C001468A068C00026D4A068634901402943EB
:105A1C00A16062480068624904F07EFA40003C9044
:105A2C003C98002817D03C98401E3C903C9800288D
:105A3C0011D03C98401E3C903C9800280BD03C98D0
:105A4C00401E3C903C98002805D03C98401E3C9051
:105A5C003C980028E7D1A0682840369B07D1404DE0
:105A6C00A96D1943A965E96D01220A43EA65A1688C
:105A7C002C9A11403A4DAA6D1A405118AA6D68D152
:105A8C0024972999C9432091F33918910A40921C03
:105A9C00AA65A268D2072E4630D1E26818239A4331
:105AAC00B3681343E3602B99725C521E534253410B
:105ABC00726823991140356C0D43776C2F43B56C8C
:105ACC003D43F16C294319432369364D1D400D4369
:105ADC0025610123DD07AA4226910ED00325AD07CF
:105AEC00AA420AD09B079A4207D0299B9B041A40D2
:105AFC002D4D2F689F43BA182A60194E326B531ED6
:105B0C009A411203337E9B03757EEF031F43B57ED0
:105B1C006B033B43F7681F4317433369002B23493F
:105B2C0002DA17311940279127990F430C49289A0B
:105B3C008A5C52003A43389E8F5D012F3AD1002D7A
:105B4C0036D007498D6D35438D65CD6D2F43CF65AF
:105B5C0030E01A43AA659BE0EDBF000890BD000839
:105B6C00640A00200024014034100240000400505C
:105B7C00C80A00200400024062BE0008FF7FFFFF3D
:105B8C0000080240F8FFFDBF8408024044090240AF
:105B9C0008E400E000E100E0E8FFFF6F5C0B002090
:105BAC00400D030002FCFF1F08270140E8FFFF7FA8
:105BBC001E9D2A43F34E756A002D05D0379F613721
:105BCC003D401543B26A2A43E568EF4F2F40174317
:105BDC00E7602569ED4F2F4026990F4327616569D2
:105BEC002F9FBD43776B2F436761656970212891A7
:105BFC008D43B76B3F012F436761002B13D03B994B
:105C0C004D05AB421ED1DF4B1B6E1D46299E354008
:105C1C000F2DA56A0CD0F0271F40F02F08D120992A
:105C2C000D43A5620EE0A36A20990B43A36209E021
:105C3C00D44DED69AD001C351C272F402099B9407F
:105C4C001943A162E168D24B0B40934215D1002756
:105C5C00CC4BDF65996D3B9A1143259A914399651D
:105C6C00002815D03F973E97CA483D903DA8FDF7B8
:105C7C0005FB00280ED072B6FEE7C24A906D36992D
:105C8C000843259988439065D06D3B990843D065AE
:105C9C0072B6FEE72C983E90BF483D903DA8FDF7AC
:105CAC00EDFA002801D072B6FEE72A983E90BB4868
:105CBC003D903DA8FDF7E2FA002801D072B6FEE750
:105CCC0022983E90B6483D903DA8FDF7D7FA0028A3
:105CDC0001D072B6FEE7B349B34D8F65CF653A98E4
:105CEC0004048D63CF630F643E464F64349888641C
:105CFC001D98C8640C651C98486508463830279078
:105D0C00FDF7E6FC002801D072B6FEE7A749802219
:105D1C000E624E62281D41C10E604E603498886040
:105D2C00269208390846143054C00846FDF7D0FCBA
:105D3C00002801D072B6FEE79D489A49C860087CDD
:105D4C0000281DD19749487446904590994B996805
:105D5C00249A11439960996811403D913D991968B5
:105D6C00012211431960196811403D9144900320A0
:105D7C004390369842903D9842A92198FEF798F8A6
:105D8C00259888490874CE613B980874487C012892
:105D9C0001D172B6FEE72598824B1874D868C16B96
:105DAC003B9C21432D9A9143C1630168824A114067
:105DBC0001608249FE3902680A4002600168C02213
:105DCC00914301605E741C741E98401E7C4A774996
:105DDC000A634E638E63C8630E644E648E64409691
:105DEC003F963E963D962698802805D0379A3E3AA7
:105DFC007448754904F0EAF96D216C480F46405C13
:105E0C00002822D16C21694A5054116B6C4A914282
:105E1C001BD10121CA02674CE3681343E360E368BA
:105E2C0013404293429A22680A43226022680A4035
:105E3C004192022146914590449043913298429070
:105E4C00419842A92198FEF733F825985749C8552F
:105E5C00086B02683B9989072091884205D0584904
:105E6C00884202D05949884205D128998A434F4922
:105E7C00896B114300E01146554A904209DD554AA1
:105E8C00904211DC4E4A904214D0534A904211D0A9
:105E9C0070E00122920790420CD04C4A904209D0FB
:105EAC004E4A904206D065E04D4A904202D04D4A8F
:105EBC0090425FD14C4A11403C4A126C0A432699DD
:105ECC008A433A4B996C11430160D96BC162596B8F
:105EDC008162464941181B9AD141072907D83B9A40
:105EEC008A40E1210A4202D03049496C01633B9A55
:105EFC00426178232D491793CA546E231693CA54C2
:105F0C000B466E335A709A70DA701A711D465A71BC
:105F1C0074231493CA540B4674335A709A701593A5
:105F2C00DA70CA556C222392895C012901D172B6B0
:105F3C00FEE725991D4AD1553B99239BD154816885
:105F4C002B4A0A4082602B4CA0420ADD2A49884227
:105F5C0012DD214988425AD02249884257D0204923
:105F6C0052E0264988424BDC0121890788424ED0F9
:105F7C00164949E00A46A2E71849884247D0104919
:105F8C0042E0C046640A00201902FEFF02FCFFDF5B
:105F9C00E7FF3F8320000014400000188000001C25
:105FAC000001002000000020000201406C090020CC
:105FBC000074004034100240FFBFFFFFFFF0FFFFF2
:105FCC00002C0140EDBF0008CBBE000800040040CF
:105FDC00FF2B0140FF4301400040014000200040E6
:105FEC000048014000440140FFFCFFFF00D4FEBF0D
:105FFC008800CEFFFF1F0040FF3F0140FF0F004015
:10600C00F649884203D0F649884200D084E1F5492C
:10601C00239A8E543B9ACA55A0420ADDF249884213
:10602C0010DDF249884219D0F149884216D0F14965
:10603C0011E0F14988420ADC0121890788420DD020
:10604C00EE4908E0EE49884208D0EE4903E0E34906
:10605C00884203D0E249884200D065E1E148806B78
:10606C002C99C841062800D9CBE03B998140572098
:10607C00014200D1C5E0DB48006C00280DD03B99F3
:10608C000902884209D03499884206D03B98C20252
:10609C00623ADD48DD4904F099F8D248806C2699C3
:1060AC000843802806D03B98C202613AD648D749AB
:1060BC0004F08CF8CB48C05D002802D1C949239A62
:1060CC0088542598C749C855086B2099884202689E
:1060DC0005D0CC49884202D0C849884205D12899BC
:1060EC008A43C049896B114300E01146C84A90426B
:1060FC0009DDC84A904211DCC24A904215D0BB4A15
:10610C00904212D006E10122920790420DD0BB4A78
:10611C0090420AD0BA4A904207D0FBE0B54A90426E
:10612C0003D0B34A904200D0F4E0BB4A1140AD4AD0
:10613C00126C0A4326998A43AA4B996C114301604D
:10614C00D96BC162596B8162B44941181B9AD14118
:10615C00072907D83B9A8A40E1210A4202D0A1497B
:10616C00496C01633B9A42619E49179BCA54169B2A
:10617C00CA546A70AA70EA702A716A71149BCA5464
:10618C00159B5A709A70DA70CA55A149884205DC81
:10619C000121890788420DD0984903E0994988422A
:1061AC0008D09249884205D09D4AA5329648974915
:1061BC0004F00CF88B482399405C012801D172B68D
:1061CC00FEE725988749C8553B98239A8854086B55
:1061DC008168944A0A40543282608D49884207DDB6
:1061EC008C4988421ADC8749884222D07F4919E0C1
:1061FC000121890788421CD08049884219D08049E6
:10620C0010E00120C202633A7F48804903F0DEFFB0
:10621C007448006C002800D031E73EE7744988428E
:10622C0007D07449884204D0774878497E4A03F0F5
:10623C00CDFF6C4B23981E54186B016A026A3B9D70
:10624C00AA4302628269F0242C94A2438261259AAB
:10625C0011432A9A91430162C1681D9A9143C1600E
:10626C00C168724A1140C160DD557149884208DC31
:10627C000121890788420DD0604988420AD05749CC
:10628C0006E05749884205D05E49884202D05749FA
:10629C00884259D125985349C855239A8D54086B77
:1062AC0042685849884201D162490A4028998A4378
:1062BC0081684260564A904205DC01229207904266
:1062CC0007D04E4A03E0494A904202D04D4A9042D0
:1062DC0002D180229143816042483146239A8654F0
:1062EC00C55540963F963E9525983D903DA8FEF7A6
:1062FC004DF8002801D072B6FEE73A48006B4449CD
:10630C00884218DD434988422BDC3E49884234D010
:10631C0036492AE00A460DE73B483C49404A03F01F
:10632C0055FF3048006B72E6D202643A3648374962
:10633C0003F04CFF92E60121890788421DD02F49BA
:10634C0088421AD02E4910E0EA02923A2E483A4975
:10635C0003F03CFF23482399405C01289AD172B684
:10636C00FEE72349884208D02249884205D0334AA7
:10637C00C83A2548304903F029FF1A482399405C54
:10638C00012801D172B6FEE716484654006B816EA7
:10639C0029430E222892914381663D963DA8042103
:1063AC000C91FDF7F3FF002801D072B6FEE70D4803
:1063BC00006B1749884207DD1649884240DC1149B9
:1063CC00884249D009493FE001218907884243D0DE
:1063DC000A49884240D00A4936E0C04600100040C5
:1063EC00001400406C090020FF3F014000400140B8
:1063FC000044014000480140FF0F004000040040F1
:10640C0000200040002C0140EDBF0008CBBE00086E
:10641C00FF2B0140FF430140FFFCFFFF00D4FEBFF8
:10642C00D914000088FFCEFF6C1C0000FFBFFFFFDB
:10643C00FF1300408FFF0FFF48C20008C409000083
:10644C00EC49884208D0EC49884205D0EB4AC83A5E
:10645C00EB48EC4903F0BAFEEB482399405C012869
:10646C0001D172B6FEE7E8484654006B816EE74AEC
:10647C001140329A11438166E549E64A0E624E623A
:10648C008E624B20179000020A6048601A98886050
:10649C00CE602E980861229848618E61CE6184206E
:1064AC0008900858002836D180200025D8490D5472
:1064BC00086890422FD10124A003D74AD168014328
:1064CC00D160D1680140429142981068204310601D
:1064DC00106820403D90469445954495022743977B
:1064EC000920400242903D9842A923912198FDF742
:1064FC00DFFC46944595449443972E9842902198FE
:10650C002399FDF7D5FCC54A1069C54908401061AF
:10651C00E006C44908602422BD48089906924250FE
:10652C00006801683B9A91430160FEF75BF8012813
:10653C001BD0B748806A002801D0FEF7CFFA3B9BEE
:10654C009903B348006882680A43826081681C9A88
:10655C00914381600168B44A0A40026001681943A2
:10656C000160FEF7B7FB002801D072B6FEE7A84821
:10657C000068AE4988420BD0AD49884208D0A54985
:10658C00884205D0349A62329D48AA4903F01EFE17
:10659C0026989F49085C012801D172B6FEE79C4AF7
:1065AC00089806991150146820682E9020683B9B1F
:1065BC00984320602498401EA1680140A160506E51
:1065CC0023900028184612D0A568A068400F9A4F57
:1065DC00395C9A4A105CC00003F09EFC3B90280189
:1065EC00400F395C954A105CC00003F095FC68279D
:1065FC008749C8536A223B982092885226980E5499
:10660C002E9820603898089A88508848844216D072
:10661C008748844213D07F48844210D0349A9332F6
:10662C007748844903F0D2FD26987949085C012803
:10663C0001D172B6FEE77648416E23910468744826
:10664C000899069A425020683B9020680125A8437F
:10665C0020602F984006A1688143A16023980028F0
:10666C00284615D0A0682E90A068400F7249095C8E
:10667C00724A105CC00003F04FFC05462E980001D6
:10668C00400F6D49095C6D4A105CC00003F044FC7E
:10669C005F49C85320980D5226980E543B982060A1
:1066AC003898089A88506148844214D060488442D3
:1066BC0011D0584884420ED0349A343250485D4937
:1066CC0003F084FD26985249085C012801D172B66A
:1066DC00FEE74F4804684E4A089B0698D050206845
:1066EC0021680125A94321600D9569078843206025
:1066FC003898D0502698165456665148406A5049DE
:10670C00496A091A64290ED84D49496A091A64293B
:10671C0009D84B49496A091A642904D84849496A75
:10672C00091A6529EBD3E6204649474D15900D52C1
:10673C00E022464814928850A81CE42213928852F6
:10674C00259888810D9888606720088040480478D7
:10675C00012C01D03F4800E03F4803F037FD0D9875
:10676C008704012C3D4C00D1C5E03D4803F02EFDC3
:10677C0002F090F93B4803F029FD3B490E86CE858B
:10678C008E854E858E840E84681C08853748488417
:10679C00CD8437484069002805D53648344988608F
:1067AC003548886048692648406A31994018304914
:1067BC0009691E9A114261D02149496A814265D208
:1067CC002B490969114259D01D49496A81425DD250
:1067DC0027490969114251D01949496A814255D258
:1067EC0023490969114249D01549496A8142DED3CE
:1067FC004CE0C0460044014000480140C409000080
:10680C00EDBF000848C200086C090020FFF0FFFF34
:10681C00DC080020003801403410024008E400E09D
:10682C00FFFFFF0000E100E0FFFF00FC0044004020
:10683C000080004034BF0008BCC20008B4C200088D
:10684C00E8090020FC060020FF7F00000000FFFF8D
:10685C0048F00108E0BC00086DC0000800F8010811
:10686C00A1BF000864C3000800000020FFFF000067
:10687C000020024023016745AB89EFCDED4B186931
:10688C00ED494A1C1A61084200D143E1E9484069CC
:10689C00C00704D0E74A50690D99884350613F20E6
:1068AC00E649886433980874087542A8FDF71EFA07
:1068BC00002801D0E2481CE0E248026A436A204604
:1068CC00FDF75CF9002813D1DE48826AC36A2046C2
:1068DC000830FDF753F900280AD1DA48026B436BF4
:1068EC0020461030FDF74AF9002801D101F014FFC1
:1068FC00D54803F06BFCD5480069000704D4D44894
:10690C0003F064FC02F0C6F8D24803F05FFC02F01E
:10691C00ABF920783899CB4A505410462030617826
:10692C004170A1788170E178C17021790171617930
:10693C004171A1798171E179C171217A0172617A18
:10694C004172A17A8172E17AC172217B0173617B00
:10695C004173A17B8173E17BC173217C0174617CE8
:10696C004174A17C8174E17CC174217D0175617DD0
:10697C004175A17D8175E17DC1750D990D02118C5B
:10698C00B54B079559538188149A9952139A995279
:10699C004188E22212929952C188159A995221216A
:1069AC000391CA00C18911929952832100914A0026
:1069BC00018A1092995241218A0041890F92995271
:1069CC008121490080890E915852188B00283BD1A7
:1069DC006420319A643A99498865CA65496E0029E0
:1069EC0000D01046954A10664842484150669B4A72
:1069FC00101F0B90006801040C9D28403940401872
:106A0C00684010600D981060259810600026304684
:106A1C00FDF7B0FB2846FDF7ADFB4296894CE068CC
:106A2C004290429808304290429806608C4803F09D
:106A3C00CDFB607C012844D18A489BE0711C8648C0
:106A4C00008B0E468142C3D22A988449086086483E
:106A5C001D9901607948406A7849496A091A379A40
:106A6C0091420ED27549496A091A914209D2734969
:106A7C00496A091A914204D27049496A091A914229
:106A8C00EAD32A987549086177481D99016100205D
:106A9C006A4908654865486A6849496A091A914211
:106AAC00CCD26649496A091A9142C7D26349496AEC
:106ABC00091A9142C2D26149496A091A9142EBD32F
:106ACC00BCE725985F490874C86801680D9A1143A2
:106ADC00016001683E220A40022A03D141680D9AE6
:106AEC0011434160574846740D9901745F4803F097
:106AFC006DFB2798FCF7E6FF002801D05C4839E0D5
:106B0C005C4803F063FB5C48FCF7DCFF00282DD0ED
:106B1C005A482FE04948406A31994018454909695B
:106B2C00394200D1B2E64549496A814200D3ADE60B
:106B3C0040490969394200D1A8E64049496A814275
:106B4C0000D3A3E63B490969394200D19EE63B4993
:106B5C00496A814200D399E636490969394200D124
:106B6C0094E63649496A8142D8D38FE6444803F00B
:106B7C002DFB444803F02AFB4296434800684349E6
:106B8C00884204D0424843496F2203F01FFB542033
:106B9C0016903D49085C0D99C9050291012800D158
:106BAC0022E10D981699384A505410688268816811
:106BBC00C907339973D025990A4033996FD18168ED
:106BCC001F9A1140012929D18168334A1140259A15
:106BDC00114381603A9901601849496A8268D20769
:106BEC005CD0164A526A521A022A17D88268D20707
:106BFC0054D0124A526A521A022A0FD88268D2070B
:106C0C004CD00E4A526A521A022A07D88268D2070E
:106C1C0044D00A4A526A521A032ADFD31A4B996D8E
:106C2C00369A11439965D96D0D9A1143D965314640
:106C3C0035E0C04600200240FAC30000E8090020FD
:106C4C0093C000080000002022BD00080004005082
:106C5C00C2BB0008C4C20008FC060020180C00507F
:106C6C001AC000082FC000081808005022BC0008E9
:106C7C00C5B80008F4C200086C090020DCB8000894
:106C8C0008C3000834BC0008640A0020002401403A
:106C9C00EDBF0008DCC10008E8FFFF7F3399826874
:106CAC00D207E14A926D40D1189B1A40259B1A439A
:106CBC00DD4B9A65C268C3683A9DAB43C360DB4B3E
:106CCC00183384681C4384602A40D94B8468002C98
:106CDC002ED5429C641C4294429C9C421AD88468D7
:106CEC00002C25D5429C641C4294429C9C4211D899
:106CFC008468002C1CD5429C641C4294429C9C428F
:106D0C0008D88468002C13D5429C641C4294429C85
:106D1C009C42DBD91698C44A1654906D3699084398
:106D2C00259988439065C34860E13698024308E092
:106D3C00C3681343C360BC48826D0D980243259809
:106D4C0082431698B84B1E549A6500294CD0BA4809
:106D5C0003F03CFAB4480068B849884208D0309A2D
:106D6C00AF32B748B74903F031FAAF480068199011
:106D7C00199881681698AC4A105C421E50425041DA
:106D8C004907339900D40146002900D02DE10D9814
:106D9C001699A54A50541998C068C0070FD1199874
:106DAC008068C00706D0199A9068A04908402599B8
:106DBC0008439060199AD0680D990843D0604296A8
:106DCC0019988068C00745D198482F30199989685F
:106DDC0001420BD0944A906D369908439065D06D62
:106DEC000D990843D06500E19248FFE0199A90682C
:106DFC008E4908400D9908439060934800680299A9
:106E0C00084221D091480068914903F085F8401C54
:106E1C0042904298002817D04298401E42904298C7
:106E2C00002811D04298401E4290429800280BD066
:106E3C004298401E42904298002805D04298401E2D
:106E4C00429042980028E7D17748407E012801D033
:106E5C0001F071FC1698744A16547E48401E916DD0
:106E6C000140329801439165D6651C23199D2B6016
:106E7C00106D7949794A7A4CC4620263416369683E
:106E8C00369A114369600699415C012900D1A6E04C
:106E9C00014624310D9A0A704A78012A00D09BE0F1
:106EAC00259A4A70C66301680A680D9CA2430A6061
:106EBC00826CC46C5460026D002A02D0446D856DE6
:106ECC006560199C4034056C1D400D9BAB40654DB5
:106EDC002F681F432F600C9B4B608568624B102DF5
:106EEC001F4600D027468F60102D00D01C46CC606A
:106EFC000B68289C23430B60406C03681E9C234248
:106F0C0003D00368329C23430360002A03D010682B
:106F1C00329B1843106008680D9A10430860199A48
:106F2C009068424908400C99084390604F4803F020
:106F3C004DF94F48806E3B90632801D901F0DBFB83
:106F4C004B49C96E329106E049490E773B9864284B
:106F5C0001D301F0D0FB46490A6F002AF4D0454812
:106F6C00C288C388444F7B431B0C9B246400434D55
:106F7C002B533F494B6FDC081B1B9A18D3087B43E0
:106F8C001B0CC8242B538B6FDC081B1B0746048976
:106F9C001B19DC083A4D6C43240C3A4D6419CA2574
:106FAC00364844533C68E508641BBD886419E50801
:106FBC00334845432D0C1B9F7D43329FED1BCC2743
:106FCC002E48C5533B98401C3B9088660E674A6719
:106FDC008B6728480460B7E70E702699C163A868D0
:106FEC00124908400C990843A860274803F0EEF8B2
:106FFC002248818A006902F08BF917988000099069
:10700C000B200190400228900D98C1041891810525
:10701C000A91C006049000211C48FE30059027916F
:10702C002091239141E0C046640A0020E8FFFF7FD5
:10703C00FFF102007CC30008C0C00008002401401E
:10704C00EDBF000890BD0008082701405C0B002034
:10705C00400D0300FFF0FFFFFBB6000849B300082A
:10706C0015320008040002400400002078B9000822
:10707C00E80900200000002088130000FC06002016
:10708C00C4090000A8FD0000E1C00008D9140000EC
:10709C000020EB493B9A88500875EA4803F096F8B3
:1070AC00E74800688821222242502098401CE6497B
:1070BC00496A814245D3E448006D002821D0401E26
:1070CC00E14908651DD1E048406DE049012800D137
:1070DC0010312A9A0A60DE49012800D110311D9A1C
:1070EC000A60411E4A1E9141D74A5165127E002A00
:1070FC00319900D10021012801D0D348C16CD2486C
:10710C000165D148006E002818D0401ECE49086693
:10711C0014D1CD48406ECD49012800D110310C9AC4
:10712C000A60411E4A1E9141C74A5166012801D08E
:10713C00C84800E0C8480068C3490866C248406AAD
:10714C0020902798401CC049496A814201D200F026
:10715C0074FDBD48416A2791006F00283ED0BF4D99
:10716C00E888E988BE4B5943090C9B225200BD4C60
:10717C00A1522646B44F796FCA08891A08183B9059
:10718C00C1085943090CC822A152B96FCA08891AFF
:10719C002C462A898A18D108B34D6943090CB34B84
:1071AC00C918CA23F15223682646DC081B1BB48875
:1071BC001B19DC086C43240C1B9D6C43BD6EFE6ECE
:1071CC00A41BCC26A74884536C1CBC6600243C67CB
:1071DC003B987867BA67A148036002E0CA20A149CE
:1071EC00095A48209F4D285E0EB2301A0A2102F02F
:1071FC006BFE4A21695A41432A8D8918EA221C9256
:10720C00A9524C21695A41436A8D8918EC22199272
:10721C00A9524E21695A4143AA8D8A18EE216A520D
:10722C005021695A4143EB8DCB182C9930936B52FA
:10723C005221695A41432B8EC918F2231E93E952ED
:10724C001699695A41436B8EC918F4232E93E9524F
:10725C005621695A4143AB8ECC18F6216C525821F9
:10726C00695A4143EB8EC918F823E9525A23EB5A59
:10727C0043434620285A1818FA23E852FC23EB5AA9
:10728C00002B02D1E823774DE8523998754B185EE4
:10729C00864203DDCE200123724D2B523A20714BD6
:1072AC00185E864203DACE2000236E4D2B522B98AB
:1072BC006C4B185E864203DAD0200123694D2B52A9
:1072CC003E20684B185E864203DDD0200023654DBE
:1072DC002B521D98634B185E864203DAD220012391
:1072EC00604D2B5242205F4B185E864203DDD2204C
:1072FC0000235C4D2B52C8235A483B93C65AA0B26C
:10730C00864206D388B2864203D8D4205549095AFE
:10731C0008E088B2864201D9002100E00121D42086
:10732C00504B1952CE234F483293C45A601E4342DD
:10733C00434190B28642339800D81846D023494A2C
:10734C00D25A571E7D427D410028339800D12846E1
:10735C004F1E7D427D410028339806D1012D06D069
:10736C00309880B2864217D325E00128F8D102204C
:10737C0036490861DE2001213A4D2952D420295A80
:10738C00EA5A32982C5A2C98285A30903B982E5AFC
:10739C00309880B286420ED2002C0CD1002A0AD131
:1073AC00002908D1022029490860DE2000212D4A3D
:1073BC0011523B98165A2B481E99405A864213D2AA
:1073CC00214A906B31994018516A81420CD3D621D5
:1073DC00244B5A5A4420185A824202D2501C214A39
:1073EC0050521949486A88631E4C3298205A401EE4
:1073FC00414241414422A05AD623E45A8442339C50
:10740C0000D00C46D2211748405A451E68426841AC
:10741C00002C339C00D10446012C07D101200B4CCD
:10742C002061DC240F4D28533B982E5A0D482E9C7E
:10743C00005B86421CD900240A48C4521AE0C0469C
:10744C00C00400208FB90008E8090020180C005077
:10745C0018080050400A0020440A002000000020B8
:10746C0088130000FC060020C4090000A8FD0000E1
:10747C00FC48C45A002C0FD1FA48329C005B0028FF
:10748C000AD1FE48405A002806D10120FC49086068
:10749C00DC200021F94C2152FE21F8483091405A51
:1074AC0002282AD1F748406C012800D1F4E0339827
:1074BC00F44A10760B98006801042A9B1840189C1B
:1074CC00214040185840EE490860EF49D164506D96
:1074DC00002800D03199EB4A116541424141516578
:1074EC00EA4A101F006801041D9B18400A9C2140A9
:1074FC004018584010600120CCE0C01E01282AD84A
:10750C00E048406C022800D1C6E03398DD4A107682
:10751C000B98006801042A9B1840189C21404018C5
:10752C005840D7490860DA49D164506D002800D022
:10753C003199D44A1165414241415165D34A101FDA
:10754C00006801041D9B18400A9C214040185840BB
:10755C00106025989EE0C9483299405A01282AD1DA
:10756C00C848406C032800D196E03398C54A107681
:10757C000B98006801042A9B1840189C2140401865
:10758C005840BF490860C349D164506D002800D0F1
:10759C003199BC4A1165414241415165BB4A101FAA
:1075AC00006801041D9B18400A9C2140401858405B
:1075BC0010603A986EE0B1493B98085A1C9C095BE4
:1075CC00884225D9AF48406C042865D03398AD4A21
:1075DC0010760B98006801042A9B1840189C2140D7
:1075EC0040185840A64908603198D0641065506D19
:1075FC00414241415165A54A101F006801041D9B81
:10760C0018400A9C21404018584010600C9841E0EA
:10761C009A49199C095B884232D29A48406C0528D9
:10762C0023D03398974C20760B98006801042A9D40
:10763C002840189E314040186840914908609621B6
:10764C00E164606D002800D031998E4C2165414277
:10765C00414161658D4C201F006801041D9D28402F
:10766C000A9E314040186840206085480D990161A0
:10767C00DC202599814C2152A05AE0521F9809E038
:10768C002A987F49086181481D99016100207D4934
:10769C00086548657B4948647A48007B002809D115
:1076AC002C9876490D5A3B980E5A0020AE4205D2C2
:1076BC000D9D12D2002500281ED010E06F49079AAC
:1076CC00885A401C885233986E4F3873724802F0B7
:1076DC007DFD387BAE420D9DECD300280CD0674964
:1076EC002E98085A3B9A895A814205D86B4802F069
:1076FC006DFD0020634908736249C86B684A8018A5
:10770C00496A8142339802D25E48007FC043C00769
:10771C0000D188E033985B490877486AC8636148B0
:10772C0002F054FD55483B99415A129A805A8142B5
:10773C0007D2524CA1525C4802F048FD3B98215AAA
:10774C00339D4E48149A805A814205D94B48815238
:10775C00564802F03BFD339DCA24484A115F1598E8
:10776C00105E814207DA1598444D2952504802F0B8
:10777C002DFD295B339D4148139A805E0AB28242EB
:10778C0008DD3E4D139829524A48114602F01EFD61
:10779C00295B339D3998394A105E323009B28842E0
:1077AC000EDA36480F9A805A434A904208D0401C51
:1077BC00324D0F9AA8523F4802F008FD295F339DC5
:1077CC001D982E4A105E323888420ADD2B480E99DD
:1077DC00405A3949884204D0401C28490E9A885294
:1077EC00339D26493B98085A498D643981420ADDFC
:1077FC002249109A895A304A914204D0491C1F4A96
:10780C00109BD152339D1D49098D643181420AD29E
:10781C001A481199405A2849884204D0401C1749EB
:10782C00119A8852339D1749086C244A8018496A6A
:10783C00814209D31349486A0864214802F0C6FC06
:10784C00002D01D001F0A2FC1E48056B1E4885429C
:10785C000ADD1E48854243DC1D4885424DD01D483B
:10786C0042E0C046FC06002001208007854244D03F
:10787C001948854241D0194836E0C046FC06002024
:10788C00180C0050E8090020581B00001808005084
:10789C0088130000B80B000055B900087CBC000828
:1078AC0060EA000092BC0008ACBC0008C6BC000832
:1078BC001CC3000834C30008FFFF000080EE360034
:1078CC004CC300086C090020FF2B0140FF43014012
:1078DC00002C01400040014000040040002000400A
:1078EC00F248854209D0F248854206D0F148F24967
:1078FC00059A02F06BFCF148056B6E6BF048854203
:10790C0005DC0120800785420FD0EE4803E0EE48ED
:10791C0085420AD0ED48854207D0289A1F3AE5489F
:10792C00E54902F053FCE548056BAC6B9720400031
:10793C00E74F3C52301B17998900785202F08CF9B2
:10794C000646204602F088F90146304602F096F8C9
:10795C00014601F095FF04463B98385A02F07CF939
:10796C00214602F02FF802F02DF906460A21329139
:10797C0002F0D2FA132109017852D8203B90385AE0
:10798C00002810D0696AD348C06A379A9532914260
:10799C000CD9CF49309A895A002907D1CD4A117296
:1079AC00401CD06207E0CA484018B0E0002829D03B
:1079BC00401EC849C862642824D3C74802F006FC9C
:1079CC0000254595449501204390389F4297469554
:1079DC0042ACC2482146FCF76BFAC0498F622F9823
:1079EC00469045954495022043904297084621467F
:1079FC00FCF75EFAB749CD6233980872086B401CED
:107A0C00086301E0B348006B0A281CD90024B04974
:107A1C003B980C524294B248C0684290429808304D
:107A2C004290429804600420309A8852AD4802F08B
:107A3C00CDFBA8490C63486B401C48633199491E27
:107A4C0088420DD80FE0A34A516B491C5163319AFF
:107A5C00521E914207D9002802D0401E9D4908634E
:107A6C0000209C494863992044009948015B99483F
:107A7C00007A9D4A964203D3002801D0012202E0ED
:107A8C0000299A4A1BD08918914A115389B2652949
:107A9C0015D300258E4F3B983D5242959048C068B7
:107AAC0042904298083042904298056002203099EA
:107ABC0078528F4802F08AFB3D538648007A4D215C
:107ACC008C008C498E428249095B03D8002801D076
:107ADC00012002E0002985481BD008187C49085376
:107AEC0080B2652815D30020794D3B99685242909D
:107AFC007B49C96842914299083142914299086088
:107B0C000320309968527C4802F060FB2819002150
:107B1C0001807A4840680028339904D0401E774988
:107B2C00486041424141DA246948005B00285DD13C
:107B3C0000295BD0714832994160E820644B1A5A95
:107B4C009B2149005B5A934228D9614D3B9EAD5B0A
:107B5C006B4EB54222D25E4E309FF65B002E1DD18D
:107B6C006A1C5B4B3B9E9A53099B5B1E9BB29D42CE
:107B7C0006D2574A099D95530022564B1A632A4642
:107B8C0000234293564BDB684293429B083342934B
:107B9C0092B2429B1A604E4B1A5A5B5A934223D2B2
:107BAC004B483B99405A00281ED0411E8AB20020F7
:107BBC00099B9A42024600D30A4645493B9BCA524E
:107BCC00429095B249480E38854205D3319A893A8C
:107BDC0038484C4902F0FAFA4148C0684290429841
:107BEC0008304290429805603948005B012813D157
:107BFC0037483B99405A4249884210D23449309A0E
:107C0C00895A00290BD142913549C9684291429950
:107C1C0008314291429908602D483B99405A31995C
:107C2C006439642200280B4600D01346294CE365C6
:107C3C00002800D00A46274882652648406A2399C6
:107C4C0088420DD92349886A496A2391002807D0B4
:107C5C00401E2049886203D1FC2000211C4A11528D
:107C6C0026202E901A48408B002800D19BE12649F3
:107C7C002E9A895C002900D095E1411E062947D82F
:107C8C004900C0467944898849008F4406004C005D
:107C9C005C00270562007C0091001C4802F096FAFB
:107CAC000020014601F036F97AE1C046004401405B
:107CBC0000480140EDBF0008CBBE00086C09002055
:107CCC00FF2B014000040040002C0140004001400B
:107CDC00FC060020E809002044C000080004005005
:107CEC0000000020F3B80008A1090100FFFF00000C
:107CFC001EB900080F27000046BC00085C0B0020D2
:107D0C00DC050000F9BD0008C0040020DCBB000845
:107D1C00F849884266D1F84802F058FA00213398A5
:107D2C0001F0F8F83CE1F54802F050FAF44800682C
:107D3C00F44988425CDDF449884267D0F3498842B3
:107D4C0064D0F34958E0F34802F040FA00F0A2FE88
:107D5C0026E1F14802F03AFA6224F048015BF0485F
:107D6C00008C814209D10020339901F0D3F86420B2
:107D7C00EA49085A0853EA490884411E88415E21A1
:107D8C00E64A50520CE1E74802F020FA6220E3493F
:107D9C00085AE349098C884226D1012000020021AF
:107DAC00DE4A115010180181416001F0EFF9F7E043
:107DBC00DD4802F00BFA6220D849085AD849098CE0
:107DCC00884211D1CA20D54A105A1599505213998C
:107DDC005052C820105A129950521499505201F016
:107DEC00D5F9DDE0D14800E0D14802F0EFF9D7E059
:107DFC00D04988420AD0D049884207D0349A74328C
:107E0C00CE48CF4902F0E2F9BD480068BC49089A57
:107E1C00069B8B50016801221C929143016000214A
:107E2C000160416019918160B949884200D0A7E096
:107E3C00C449C868C44A1040C86002203B90042062
:107E4C0032902A983090199D24E03B988140219FD4
:107E5C003868084338601C20329B1840299B8340AB
:107E6C00E80880003818046A9C430462B8688843A8
:107E7C00B860786890437860F8688843F8601E981A
:107E8C00851C3298083032903B98001D3B903098FE
:107E9C00103030901C9EAE403146289801403BD0AB
:107EAC0030980838369A1040299A824003202B4685
:107EBC008343A64CE3181C6E144211D16033A44FBB
:107ECC003C688C433C607C688C437C609F4F3C6876
:107EDC008C433C607C688C437C60196891431960CE
:107EEC003B99891E8840219C21680143216032996D
:107EFC00091F18220A4029999140EA089200A218F9
:107F0C00136A8B431362A1688143A1606168B1431A
:107F1C006160E1688143E160681C0D2829D0401E36
:107F2C0002221E908240104628990840A7D01821A2
:107F3C00309B1940299B8B4003212C468C43834F4B
:107F4C003C19276E1F4200D07FE76034804E3768A3
:107F5C00874337607768874377607C4F3F688743F8
:107F6C007A4E376077688743776020689843206043
:107F7C006BE7049877490860BFF34F8FBFF36F8F9F
:107F8C008C205F49199A0A5008980A5088200A5088
:107F9C0080200A54CA6661490869898A01F0B8F9D7
:107FAC0000205E4948836C48007D002801D1FFF712
:107FBC007CF84520C10068483B914058042801D802
:107FCC00FFF766F8074627256348405D329001208D
:107FDC001E90C443B81E3090044000265F4A03E054
:107FEC00B61CB44200D1BDE05B488019415D5140E4
:107FFC008AB25208C9071DD059494A405308D107C3
:10800C001BD15A08D9071DD055494A405308D107EE
:10801C001BD15A08D9071DD051494A405308D107E2
:10802C001BD15908DA071DD04D4A51404A08C907DF
:10803C001BD11CE05308D107E3D049494B405A08E7
:10804C00D907E1D15308D107E3D045494B405A0831
:10805C00D907E1D15308D107E3D041494B40590826
:10806C00DA07E1D14A08C90701D03D494A40282323
:10807C00C15C51404808C9071DD0394948404108E6
:10808C00C0071BD14808C9071DD0354948404108D5
:10809C00C0071BD14808C9071DD0314948404108C9
:1080AC00C0071BD14808C9071DD02D4948404208BC
:1080BC00C00795D01BE04108C007E3D028484140D9
:1080CC004808C907E1D14108C007E3D02448414022
:1080DC004808C907E1D14108C007E3D02048414016
:1080EC004808C907E1D14208C00700D178E71C480D
:1080FC00424075E739300000B2BF0008F2BB0008FF
:10810C00DC080020FF4B0040004C00400080004089
:10811C0000380140D9B20008C7BF0008FC06002097
:10812C00E80900200CBC0008D4C20008DCBF000821
:10813C00A6B800080044004000480040EDBF00080D
:10814C0058BB000834100240FFBFFFFF001802406C
:10815C008018024080E100E0C0040020FFFF000016
:10816C0001A00000F80742D0FD480019405D4240D4
:10817C0090B24008D1071DD0FA4948404108C007C9
:10818C001BD14808C9071DD0F64948404108C00713
:10819C001BD14808C9071DD0F24948404108C00707
:1081AC001BD14808C9071DD0EE4948404208C007FA
:1081BC001BD11CE04108C007E3D0EA484140480805
:1081CC00C907E1D14108C007E3D0E648414048085F
:1081DC00C907E1D14108C007E3D0E2484140480853
:1081EC00C907E1D14208C00701D0DE484240791CE2
:1081FC0048424841DC4C3099615C3D196D1E2D782C
:10820C002D02691892B29142339900D1014601298D
:10821C0003D1D64801F0DAFF25E0D548018B329D19
:10822C004A1B50425041002D339A00D00246002A7E
:10823C0019D093204500CA4A3095329850558B205E
:10824C00850000201C955051D25C102A12D0062AB1
:10825C001AD0032A25D1329A002A2BD0914229D048
:10826C008620019960E00020BD493B9A8850087532
:10827C00FEF716FF3298002828D0814226D003271B
:10828C000B2186261E9AAAE0329800282DD0814216
:10829C002BD0359828308621B14A115402210B205D
:1082AC00C7E0AF48309940181E99817026994A4012
:1082BC0042703EE0637921790902CA1811467E3971
:1082CC007C25ED43A94222D203212CE0617920794F
:1082DC000002421810467C387A23DB430327902691
:1082EC00984228D21E9A394679E0E178A0780002AB
:1082FC0040189C2800D395E08D229200984B9A58F8
:10830C00125C022A72D0002A77D19A4888E0E17870
:10831C00A47824026118521814469D3C9B25ED4309
:10832C00AC4218D2022100988D4A309BD218917021
:10833C005070032782E0E378A07832900002199302
:10834C00C418151928469D389B22D24390421BD243
:10835C0002211E9A43E0824D309C2C195B00A370C5
:10836C0003236370359B2A33EB184C00804D2C197A
:10837C00255C5D7025186D781D70801C9B1C491C3C
:10838C009142F5D3C71C59E06000794A1018472276
:10839C00D200734B9F588D2292009A582F3309E0CC
:1083AC001E7806705E1E36784670801C9B1C641C02
:1083BC00AC4208D2165D002EF7D0022EF0D13E88CA
:1083CC00002EEDD1F1E7F448309A8018199AC2705A
:1083DC00329A8270369A4270042200262D9FEE4803
:1083EC008018309A86548018417027E04722D200BA
:1083FC00E94B9A581288002A11D042006079E34B5D
:10840C0098549A1823795370E34A309C12191371BB
:10841C00D170002191702D995170052109E0E1482E
:10842C0001F0D4FE359828308621DB4A1154022005
:10843C000146D94A5218309BD0544F1C39461E98CD
:10844C0081433A460240D448309BC3180C46D04D69
:10845C0003E09B1CA41E00D18EE0187868404508F0
:10846C00C0071DD0CB4845406E08E8071BD17508E6
:10847C00F0071DD0C74845406E08E8071BD17508AA
:10848C00F0071DD0C34845406E08E8071BD17008A3
:10849C00F5071DD0BF4D68404508C0071BD11CE037
:1084AC006E08E807E3D0BB4846407508F007E1D1F9
:1084BC006E08E807E3D0B74846407508F007E1D1ED
:1084CC006E08E807E3D0B34846407008F507E1D1E1
:1084DC004508C00701D0AF4845405E786E40700833
:1084EC00F5071DD0AB4D68404508C0071BD1680887
:1084FC00ED071DD0A74D68404508C0071BD1680883
:10850C00ED071DD0A34D68404508C0071BD1680876
:10851C00ED071DD09F4D68404508C00799D01BE062
:10852C004508C007E3D09B4845406808ED07E1D1FA
:10853C004508C007E3D0974845406808ED07E1D1EE
:10854C004508C007E3D0934845406808ED07E1D1E2
:10855C004508C00700D17CE78E48454079E7C04606
:10856C00C004002001A00000E7040020FAC00008AD
:10857C00FC060020A0C30008002A43D086484018FF
:10858C003099405C4540A8B24008E9071DD08149AC
:10859C0048404108C0071BD14808C9071DD07D4978
:1085AC0048404108C0071BD14808C9071DD079496C
:1085BC0048404108C0071BD14808C9071DD0754960
:1085CC0048404508C0071BD11CE04108C007E3D058
:1085DC00704841404808C907E1D14108C007E3D0C1
:1085EC006C4841404808C907E1D14108C007E3D0B5
:1085FC00684841404808C907E1D14508C00701D087
:10860C0064484540290A644CE019309A8554801816
:10861C00417022982E996054BB1C1C98235098B220
:10862C00424242412068014680314C68202C339CE8
:10863C0000D11446002C30D10A78012A2DD00546E1
:10864C00543584686B800022CA602B80524B309D5D
:10865C005B190365039B4B60436E249DAB420DD1AC
:10866C001A9B9C4203D10369002B514B00D0514BF8
:10867C000A7043670068083002990BE01A9B9C4211
:10868C0003D10369002B484B00D0484B0A70436759
:10869C000068269902680A43026000203E4D3B990F
:1086AC0068506221394C615A334B1A8C891A4A42F0
:1086BC004A41602162522875DA835C20205A0028D6
:1086CC0001D1FEF7F2FCFC21304A1E9B5352E821EB
:1086DC005052294838498162FEF7E7FC2F4801F0D7
:1086EC0075FDBFF34F8F234914392D480860BFF334
:1086FC004F8F00BFFDE7234A1068C108401A9188CC
:10870C0040181060C00820494843000C1B9948438E
:10871C001949C866FEF76CFC19481830144A51699F
:10872C0001435161506915480069000701D4FEF7F7
:10873C00E6F8FEF7E9F81048406A199B06E00E4986
:10874C00496A091A032901D3FEF744FB19990968F0
:10875C00C90701D0FEF77EFB19998968C907EED1CC
:10876C009968074A11400D9A11439960E7E7C04692
:10877C000020024020ED00E0E80900200004005039
:10878C00E8FFFF7F00000020C4090000FC06002069
:10879C00FFFF000001A00000C004002001B300088E
:1087AC000400FA05BCC30008294E00080FB70008E6
:0C87BC00CD4D00084BB30008E093040012
:1087C8000248416A491C41627047C046E8090020D6
:1087D800F0B583B03848001F0568384A1468206827
:1087E80004260190304041424141106C1C23034053
:1087F80037469F40384602952840424242410A4344
:1088080030D0009401200226019D2A463240514270
:1088180051419E40029A1642074600D00F46002F4B
:1088280032D008210D4069426941DA40120700D56B
:108838000846002826D124200021204C2154009AE3
:1088480010680E21884310600120014699401A4B98
:108858001A680A431A60E06325216054616B002995
:108868000ED10FE02068800602D42068B043206053
:1088780011490868384308601048016B002901D085
:108888000E48884703B0F0BD2346206880060B4A8F
:1088980006D418680A21884318602520012111543C
:1088A8002420002111540449086830430860D16A23
:1088B8000029E5D1E6E7C04604000240C80A0020C6
:1088C800F0B583B06E4D286801680291EF21CC00A5
:1088D80047686C49884204D06B486C49224601F0CD
:1088E80077FC6869042806D0082804D0621C66480A
:1088F800664901F06DFC0223384618404142414167
:1089080002981840424242410A4308D1A86DC00665
:1089180003D48834A86D2043A865286803600193B0
:108928000125042038404242424102984007284627
:1089380000D510466E0201280AD10820384043426B
:10894800434102980007284600D5184600282FD131
:108958004B49886DC00602D4886D304388650B6822
:10896800D8680005800F1ED14548807E00281AD19E
:108978001868000717D59868400709D458680C216B
:1089880088435860FF200230424C2168814307E049
:108998003B48846D20212143816504465C34C16DC8
:1089A8000120084320603A48012101670C20186023
:1089B800802338461840444244410298000628461D
:1089C80000D52046002807D1012000042C4CA16DB9
:1089D8000143A1652068036001231C023946214038
:1089E800484248410299C905294600D5014600294F
:1089F80006D15804224A916D0143916510680460BC
:108A0800394631404842484102993142294600D00E
:108A18000146002906D19804194A916D01439165D0
:108A280010680660102239461140484248410299B0
:108A3800C906294600D50146002911D11048046805
:108A4800006B002802D0E068800708D098020C4E1E
:108A5800B16D0143B165F06D01990843F06522607D
:108A6800580307407A427A410299890401D403B035
:108A7800F0BD1500FBD102490968086003B0F0BDDC
:108A8800640A002000240140EDBF000890BD0008E2
:088A9800E8090020BC0A0020DF
:108AA000F0B581B06A4801F097FB6A486A4D2946E3
:108AB0005CC85CC15CC85CC15CC85CC15CC85CC1B2
:108AC000482001262E5468206864286C401C2864C5
:108AD000624F7868002806D538460838604901603A
:108AE0006049016078687D20C1005F48426A521881
:108AF00033043C681C4215D0446A944218D23C6846
:108B00001C420FD0446A944212D23C681C4209D0E5
:108B1000446A94420CD23C681C4203D0446A94429A
:108B2000E7D305E03A68514B5C1C3C601A4268D0C0
:108B30007968C90702D07968B14379603E218164C0
:108B4000067406756846FBF7D7F8002800D0FEE7E4
:108B50000CCD474C2046083DFBF716F80028FED107
:108B6000AA68EB6820460830FBF70EF80028FED113
:108B70002A696B6920461030FBF706F80028FED101
:108B8000AA69EB6920461830FAF7FEFF0028FED1EB
:108B90002A6A6B6A20462030FAF7F6FF0028FED1D9
:108BA000AA6AEB6A20462830FAF7EEFF0028FED1C9
:108BB0002A6B6B6B20463030FAF7E6FF0028FED1B7
:108BC000AA6BEB6B20463830FAF7DEFF0028FED1A7
:108BD0002A6C6B6C20464030FAF7D6FF0028FED195
:108BE000AA6CEB6C20464830FAF7CEFF0028FED185
:108BF0002A6D6B6D50342046FAF7C6FF00281DD051
:108C0000FEE7426A5118B2043B68134290D0436AAF
:108C10008B428DD23B6813428AD0436A8B4287D203
:108C20003B68134284D0436A8B4281D23B68134233
:108C300000D17DE7436A8B42E6D379E7F007796894
:108C400001437960786800F015F801B0F0BDC046C6
:108C5000F6BC0008CCB100086800002010200240DB
:108C600023016745AB89EFCDE8090020FAC3000076
:048C700000F0010807
:108C7400F0B588B0A3490A78A34802704A784270D4
:108C84008A788270CA78C2700A7902714A7942710C
:108C94008A798271CA79C2710A7A02724A7A4272F4
:108CA4008A7A8272CA7AC2720A7B02734A7B4273DC
:108CB4008A7B8273CA7BC2730A7C02744A7C4274C4
:108CC4008A7C8274CA7CC2740A7D02754A7D4275AC
:108CD4008A7D8275CA7DC2750A7E02764A7E427694
:108CE4008A7E8276CA7EC2760A7F02774A7F42777C
:108CF4008A7F8277C97FC17784490A782023C25446
:108D04004A782123C2548A782223C254CA7823235E
:108D1400C2540A792423C2544A792523C2548A7935
:108D24002623C254CA792723C2540A7A2823C25458
:108D34004A7A2923C2548A7A2A23C254CA7A2B2310
:108D4400C2540A7B2C23C2544A7B2D23C2548A7BEF
:108D54002E23C254CA7B2F23C2540A7C3023C2540C
:108D64004A7C3123C2548A7C3223C254CA7C3323C2
:108D7400C2540A7D3423C2544A7D3523C2548A7DA9
:108D84003623C254CA7D3723C2540A7E3823C254C0
:108D94004A7E3923C2548A7E3A23C254CA7E3B2374
:108DA400C2540A7F3C23C2544A7F3D23C2548A7F63
:108DB4003E23C254C97F3F228154554A117840232F
:108DC4000793C15451784123C154917842230693A7
:108DD400C154D1784323C154117944230593C15418
:108DE40051794523C154917946230493C154D179CF
:108DF4004723C154117A48230393C154517A492318
:108E0400C154917A4A230293C154D17A4B23C15459
:108E1400117B4C230193C154517B4D23C154917B4D
:108E24004E230093C154D17B4F23C154117C502550
:108E34004155517C5123C154917C52240155D17C1C
:108E44005323C154117D5423C154517D5527C15519
:108E5400977D56214754D27D5727C25507682D4A1E
:108E6400176187889782C788D782078917834789BC
:108E7400178587895785C7899785078AD785478A3C
:108E84001786878A5786C78A9786078BD786478B24
:108E94001787878B5787C78B9787078CD787478C0C
:108EA400079E9753878C069E9753C78C059E9753AE
:108EB400078D049E9753478D039E9753878D029E7B
:108EC4009753C78D019E9753078E009E9753468EE6
:108ED4005653858E1553C48ED452038F5352418FEB
:108EE4005823D152818F5A23D152C18F0A4B1984EE
:108EF400002902D05E2101235352C06C506008B097
:108F0400F0BDC04600F001086800002020F0010810
:0C8F140040F00108FC060020E8090020E5
:108F2000F0B583B00D460190914801F055F9914F8D
:108F300038697969904E03C6388B3080388D7080DF
:108F4000788DB080B88DF080F88D3081388E70814A
:108F5000788EB081B88EF081F88E3082388F708232
:108F6000788FB082B88FF082F88F30834020385AE3
:108F700070834220385AB0834420385AF083462008
:108F8000385A30844820395A71844A21795AB18438
:108F90004C21795AF1844E21795A31855021795AE0
:108FA00071855221795AB1855421795AF18556211A
:108FB000795A31865821795A71865A21795AB1865F
:108FC0006E4C083E002D02D12146203101E0394689
:108FD0006431098801253554F18768207064306C4C
:108FE000401C30640198002804D0654801F0F4F872
:108FF0007868F064634F7868002806D538460838EA
:10900000614901606149016078687D20C000616A42
:1090100009182A043B68134215D0636A8B4218D2A0
:109020003B6813420FD0636A8B4212D23B681342F3
:1090300009D0636A8B420CD23B68134203D0636A47
:109040008B42E7D305E03968514A531C3B6011421B
:1090500068D07868C00702D07868A84378603E205E
:10906000A0642574257502A8FAF746FE002800D0F2
:10907000FEE70CCE474C2046083EFAF785FD002857
:10908000FED1B268F36820460830FAF77DFD00286B
:10909000FED13269736920461030FAF775FD002859
:1090A000FED1B269F36920461830FAF76DFD002849
:1090B000FED1326A736A20462030FAF765FD002837
:1090C000FED1B26AF36A20462830FAF75DFD002827
:1090D000FED1326B736B20463030FAF755FD002815
:1090E000FED1B26BF36B20463830FAF74DFD002805
:1090F000FED1326C736C20464030FAF745FD0028F3
:10910000FED1B26CF36C20464830FAF73DFD0028E2
:10911000FED1326D736D50342046FAF735FD0028CC
:109120001DD0FEE7616A0818A9043A680A4290D087
:10913000626A82428DD23A680A428AD0626A824268
:1091400087D23A680A4284D0626A824281D23A68FF
:109150000A4200D17DE7626A8242E6D379E7E807F6
:109160007968014379607868FFF784FD03B0F0BD4A
:109170000CBD0008FC06002068000020E809002063
:1091800086C000081020024023016745AB89EFCD5F
:08919000FAC3000000F0010821
:10919800F0B581B0544801F01BF801252902534865
:1091A800415A534E3184E021415AB184E221415A57
:1091B8007184E421415A3185E621415AF184212103
:1091C800C900415AF18583214900415A318641211C
:1091D8008900415A718581214900405AB085454F1F
:1091E8007868002806D5384608384349016043495D
:1091F800016078687D20C1004148426A52182B04FA
:109208003C681C4215D0446A944218D23C681C42FF
:109218000FD0446A944212D23C681C4209D0446A76
:1092280094420CD23C681C4203D0446A9442E7D36F
:1092380005E03A68334B5C1C3C601A4230D07968D0
:10924800C90702D07968A94379603F218164057410
:1092580005756846FAF74CFD002804D02A4800F046
:10926800B7FF01B0F0BD326A736A284C2046FAF79E
:1092780087FC00280FD1B26AF36A20460830FAF753
:109288007FFC002807D1326B736B10342046FAF745
:1092980077FC002820D01E4800F09AFF01B0F0BDEE
:1092A800426A5118AA043B681342C8D0436A8B42E9
:1092B800C5D23B681342C2D0436A8B42BFD23B68D7
:1092C8001342BCD0436A8B42B9D23B681342B6D032
:1092D800436A8B42E7D3B2E7E807796801437960CC
:1092E800786801B0F0BDC04664C30008FC060020E1
:1092F800000000201020024023016745AB89EFCD14
:10930800E8090020FAC3000093C0000800F801082B
:0493180022BD00086A
:10931C00F0B58DB0024608466538444244410846D3
:10932C006F3843424341234303D102206F2903D1B9
:10933C0004E001206F2901D0652901D10A3000E039
:10934C0009309A4D6A609A4E35600127BA023C0387
:10935C0065290492059406D06F2902D103214A0293
:10936C0001E000221446AC602A610021002B00D1E0
:10937C007903E96000F080FC8E4B002202F090F83B
:10938C0000F032FC2A688C498A42069009DD8B4930
:10939C008A420CD08A498A4209D08A498A4206D02C
:1093AC0046E089498A4202D088498A4240D18424C5
:1093BC002859002846D1802000262E54286881493F
:1093CC00884233D1B8038449CA680243CA60CA6868
:1093DC0002400892089808683843086008683840CA
:1093EC0007900C970B960A9602200390099009207F
:1093FC0040020890079805200007029008A90191E7
:10940C00FAF756FD0C970B960A9703980990049857
:10941C00089002980199FAF74BFDFF2000066F495E
:10942C000A6882430A60F8066D490860604E09E0DC
:10943C003A0249326648674900F0C8FE842428592C
:10944C000028B8D02420285128680168B94301604D
:10945C00FBF7C8F8012827D0A86A002801D0FBF731
:10946C003DFBB903286882680A438260F90382686D
:10947C008A43826001685B4A0A400260F9054268CF
:10948C000A434260B90602680A430260FF242106BF
:10949C0042690A4006990A434261016839430160F6
:1094AC00FBF718FC002801D072B6FEE731680A46BB
:1094BC0080329068202809D18B680598834202D1AC
:1094CC000869002802D01078012803D14C4800F01C
:1094DC007DFEFEE70D465C3500200690C8661770D1
:1094EC002C806C8027368E65002B0AD03E07B34249
:1094FC000BD03E03B3420DD10E69002E0DD13A4C68
:10950C000BE00E69002E07D107E00C69002C03D08C
:10951C003F2402E0A88001E07F24AC80D0602224AC
:10952C0094600E68B4683C43B460380204907C07C5
:10953C00486EA04202D1A889FF280DD90598834214
:10954C0002D1086900282DD02B4B069C049D147069
:10955C000B672035334610E00598834202D1086929
:10956C00002821D0224D069C3346083314700D6719
:10957C0030680499084330603D070D4A2620145486
:10958C004720C0001F4911508D2080001B491150ED
:10959C001868284318609484D46114841C32947124
:1095AC000DB0F0BD134BD0E7104DDCE7DC0800200C
:1095BC00C004002000000C40FF4B0040004C004059
:1095CC00008000400038014000440040004800404A
:1095DC00EDBF000813C100083410024018E400E08D
:1095EC0000E100E0FFFF00FCFF010000A94F0008B4
:1095FC006D4E000807B400089DB30008700B0020E6
:08960C0044BD0008060A00201D
:10961400F0B58AB098480168CC6908680990486830
:10962400012007900007069088680890230753D00C
:109634000698401C089A104001252A021646203636
:10964400099F3E40064347D03A4056425641E207FE
:10965400079A00D03246002A05D10D628C22864F2B
:10966400BE582E43BE50089A15406A426A41A60766
:10967400079E00D51646002E08D102220A628C22CB
:109684007D4EB658042737437B4EB7506A426A4131
:109694006507079D04D4002D04D0002B0CD41BE0D7
:1096A4001500FAD104220A628C22734FBD58022697
:1096B4002E43BE50002B0FD5421E9041099A9206AC
:1096C400079A00D40246012A06D1082008628C2297
:1096D400694DAB580343AB500125E80504902005C0
:1096E40013D50898049A1040AA06099B1A4010182A
:1096F4000BD0E8020862882020225F4B1A50842095
:109704001A505E4805755E4A855403952020274605
:10971400059007401ED00898069A1040099A059BA8
:109724001A40024316D04520C000544A13588825D5
:10973400514E7559222D00D094E0FE2B00D991E0B2
:10974400D3184D6A27269D554D4B039DD554135868
:109754005B1C1350802326461E402ED00898049A82
:109764001040099A1A40024327D0444800688422D2
:109774008258212A14D1024656321588002D0FD062
:1097840005680195056D02952D780092019A956200
:10979400029A551C0565009A1088401E108007E047
:1097A400006802689A430260026840251543056018
:1097B400324D23200001039A2A5402934025099A2A
:1097C4002A4050425041620600D50790079800286D
:1097D4000DD10868A84308608420274B059A1A50C5
:1097E400284800220270882022241C505A678C22A8
:1097F4002148805800282AD0882422201E4B185142
:10980400002F09D0089B079106991940099F059BD1
:109814001F400F4307991CD1002E18D0089B049AAF
:109824001340099A029E32401A4310D00A68AA4390
:109834000A608421104B059A5A50185126200F496A
:1098440000220A5423200001039C0C545A670AB0D6
:10985400F0BD8869082303438B61002006498850C2
:109864000AB0F0BD8869082202438A618023264633
:109874001E40A2D072E7C046DC080020C0040020CD
:0898840031020000E60400209F
:10988C000122D20703004B403AD430B4431A01D220
:10989C00C01AC9184B004400240EFF2C29D0002CF0
:1098AC0024D01B0E20D0E31A182B1DDC0902114307
:1098BC00C40D000210435D4219350A00AA40D209BA
:1098CC00D940451801D36D080234013CE405280A3F
:1098DC000121C9072D062A438A4160414100090E26
:1098EC00FF2901D3C00DC00530BC7047C00FC007A5
:1098FC00FAE74202F8D07F2000010C300005F3E7B4
:10990C00A4465140431A02D25340C01AC9184B0006
:10991C00090211431B0E4400240EFF2C41D0002BD6
:10992C0010D05B421B19012B10D322D1C30D400266
:10993C00401A10D3DB050100400AC905914158417A
:10994C00644670472442FBD10020F9E7C30D400266
:10995C004900401AF4D0002101314000FCD38C4264
:10996C0004D95B1ADB05400AC018E9E7180AC007DE
:10997C00E6E7192BE4D801330C00D940DC414C400C
:10998C00012C4941C30D00021043441A01D4A40018
:10999C006408013BDB05200A2406944158416446C7
:1099AC007047FF2B01D04102CAD07F2000010C3040
:0499BC000005C5E7F6
:1099C0000122D2075140014B18470000919800082E
:1099D00030B405004D400124E407254042004B000F
:1099E000120E32D01B0E3CD0FF2A33D0FF2B3FD0BB
:1099F000D21800022043000A09022143090AC4B216
:109A00004C43000AC3B24B43000A4843210A5B1887
:109A1000190A091801D44900013A080A7F3A2ADBD9
:109A2000FE2A0FD2D2051C43240601D00124214373
:109A3000C9B280295041802901D140084000284303
:109A400030BC7047FF20C005F9E71B0EFF2B0AD082
:109A50002800F5E7400206D1FF2BF3D1490202D1DD
:109A6000F0E7FF2AF4D17F2000010C300005E7E782
:109A70004902F8D1E6E743020132E9D15B12023331
:089A8000E6D9D805E4E7C04671
:109A880030B405004D400124E407254042004B0056
:109A9800120E26D01B0E34D0FF2A2DD0FF2B35D026
:109AA800D21A000220430902214343084908A00DA5
:109AB8005B1A02D2013A5B005B185B008B4200D351
:109AC8005B1A4041F9D37F3222DDFF2A06D2D20544
:109AD800C91A8B425041284330BC7047FF20C0054B
:109AE800F9E71B0E03D0FF2B12D1490210D07F20BB
:109AF80000010C300005EFE74002F8D1FF2BEDD153
:109B0800F5E7FF2AEAD14002F1D1E7E74902EED1B1
:049B18002800E1E759
:109B1C0002000A43520008D0884204D140000121BF
:109B2C000906C84201D90020704701207047C04681
:109B3C00012212064300DA4211D84B00DA420ED849
:109B4C0002000A43520008D003D2884280410130FF
:109B5C0070478142804101307047012070470020DE
:049B6C007047C04638
:109B7000012212064300DA420FD84B00DA420CD819
:109B800002000A43520008D003D281428041404281
:109B90007047884280414042704700207047C0466D
:109BA000012212064300DA420FD84B00DA420CD8E9
:109BB00002000A43520008D003D28842804140424A
:109BC0007047814280414042704700207047C04644
:109BD00041000DD2090E7F390AD449421F3105D404
:109BE00000020122D2071043C8407047C8177047CF
:049BF000002070479A
:109BF4004A0010D2520D03231B02FF33D21A0AD497
:109C040052421F3209D4400DC90208430123DB0725
:109C14001843D040704700207047D0177047C046A3
:109C2400420017D2120E7F3A14D480231B06202A36
:109C340006DA52421F3200021843D0400021704716
:109C440052423F3209DB010219430800D041D1409E
:109C540048407047002001007047D017010070474A
:109C64009D2201000AD002D4013A4900FCD5D20554
:109C7400080A0906494100D3012950417047C046EA
:109C840042221201033A010007D002D4013A00181B
:0C9C9400FCD51205C30A40059918704762
:109CA000BD22094210D003D4013A00184941FBD526
:109CB000D2050128804101300143080A09064941C3
:109CC00000D301295041704700490847659C0008AE
:109CD0004B1801225205DA4217D25B0D0722D2013E
:109CE0009B1A0FD9FF2B13D2DB05CA0FD2071343E0
:109CF0000903020D1143490AC200524100D9013142
:109D0000C8187047C80FC007704706D1002804D193
:109D1000C80F0002FF30C00570470123DB070A00AF
:109D2000C900400F084398431A4010435B0A184388
:049D30007047C04672
:109D3400F0B581B00A464149C30D5C1EFD2C58D8CC
:109D4400FD24E443D50DFF3DA54252D306460E4003
:109D5400491C0140964260D90091DCB20123DD0523
:109D6400002C03D0691E0840284309E0AE4206D205
:109D74009F05641E7000BE420646FAD300E03046DA
:109D8400D10DCEB2002E03D0691E0A402A4308E04A
:109D9400AA4206D29F051146761E4A00B9421146D0
:109DA400FAD3B4420ADD811A02D4904201D109E007
:109DB4000146641E4800B442F5DC3446861A03D4D6
:109DC400904202D1009A11E00646AE4206D29905AD
:109DD400641E70008E420646FAD300E03046002C22
:109DE4001FDD611E009A8018C9054218104601B093
:109DF400F0BD4500124CA5421BD25500AC42F5D92A
:109E040006460E40FF24E5050E4CAE4213D0002E4C
:109E14000BD10A420246E9D10DE000D001460A46C0
:109E2400E4E7191BC8400021DCE70A4003D0AA423A
:109E34008ED10246DAE72246D8E7C046FFFFFF7F0D
:089E4400010000FF0000C07FD7
:109E4C00C10DC9B24A1EFE2A19D27E2903D8002898
:109E5C0013DA104870479529FCD87F390C4A0A410F
:109E6C000240134603D5094B5B1CCB40D3188840EA
:109E7C00400200D01A461046704700207047002957
:109E8C00E8D10121C90708407047C046FFFF7F0099
:089E9C00000080FF000080BF00
:109EA40030B5514343435C18010C130C0D005D4362
:109EB400641992B2514380B242430D0C0904521802
:109EC40065415843010C00048018694130BDC04607
:109ED400CA1751408B1A17D0C1174A4094464840BC
:109EE400411A48081A0000E052008242FCD90020BE
:109EF40000E05208914200D3891A40419A42F8D1B5
:109F040062465040801A704710B500F07DF810BDCD
:109F140007B5FFF7DDFF0EBC4243891A00BDC046FA
:109F24000A0015D00300400800E052008242FCD928
:109F3400002000E052089B1A06D340418A42F9D11E
:109F4400704752089B18F8D200188A42F9D170471A
:089F540010B500F059F810BD32
:109F5C0038B504004D42FFF7DFFF4543611938BDAA
:109F6C00002B09D1002907D110B51100FFF7F0FF24
:109F7C000A000021002310BD70B400240125ED0758
:109F8C00002B07D1002905D0834203D213000022F5
:109F9C002C0000250026A419994200D1904212D918
:109FAC0092185B4103D2EE076D086408F3E7DE07F5
:109FBC005B08520892190126F6079B1903E0DE078D
:109FCC005B0852089219801A994103D364416D4180
:109FDC00F5D30FE024196D410AD2DE075B08520855
:109FEC00921980185941F5D364416D41E7D301E0D2
:109FFC008018594102000B002000290070BC7047EA
:08A00C00002000217047C0464E
:10A0140003490868002800D0704702480860704768
:08A02400400B0020480B002056
:10A02C007F2805D8034A125C0348405C10407047F7
:0CA03C0000207047E4C30008B5C1000814
:10A048007F2805D8034A125C0348405C10407047DB
:0CA0580000207047E4C30008B5C10008F8
:10A06400411C02780130002AFBD1401A7047C046D7
:10A07400002A03D0013A8B5C8354FBD17047C0465D
:10A0840000220B0011001A00002A02D0013A815468
:04A09400FCD1704744
:10A09800F0B581B00022002933D00378002B30D0EE
:10A0A800032302469A4316680024E5438707FF0EF8
:10A0B800BD40ED43354306461E4071180429009300
:10A0C8000AD3124EAF19104BAB433B4204D1091FC0
:10A0D8005568121D0329F5D82B060DD02B041B0E2D
:10A0E80007D02B021B0E06D02B0E009C04D0042494
:10A0F80002E0012400E002248C4200D30C46101A2E
:10A108000219104601B0F0BD80808080FFFEFEFE7F
:10A11800F0B581B004467F20C605002C00960FD00C
:10A12800E11722464A40571AC6050A4DF80704D0D7
:10A1380029683046FFF748FC06462D1D7F08F5D1F3
:10A1480000983146FFF79CFC002C00D4304601B043
:08A15800F0BDC046A0B20008F2
:10A16000F0B503AF93B06E46F51D2135F41D3934BB
:10A1700074613362F261F160306100F0FDFEB06045
:10A18000C21D07218A436946B1616946881A706019
:10A190008546F41D1D34002124222046FFF776FF5A
:10A1A0000B487169F2680A6048600A4828603069A3
:10A1B0002862B06868617068E8602046F169326AB8
:10A1C00000F01EF8B1698D46FC1F053CA546F0BDA8
:08A1D0007FB80008FFFFFF7FCC
:10A1D80083B010B581B0044603A80EC005480068D6
:10A1E80003AA0092214601F073FA01B010BC02BC28
:08A1F80003B00847640B0020CE
:10A20000F0B59FB014460F46002115900160012063
:10A2100002020C92460282020392C20202920322BE
:10A220000A92920205920203179242030792820356
:10A2300004920090C00316900891C84301900F96B5
:10A240003978252908D0002901D100F060FE7F1C53
:10A25000159801F0E4F9F3E7FF1C089BB81E057898
:10A260002A46203A102A2BD880219200184602A3B1
:10A270009A5803469746C046BDA20008DDA20008D2
:10A28000DDA20008D7A20008DDA20008DDA20008B8
:10A29000DDA20008C9A20008DDA20008DDA20008B6
:10A2A00007A30008CDA20008DDA20008D1A2000883
:10A2B000DDA20008DDA20008D5A2000840210AE0C6
:10A2C0005E2D179907D009E0169904E0202102E0DD
:10A2D000102100E031460B437F1CBFE77F1E29465B
:10A2E0003039C9B20929139419D800240A216143CD
:10A2F0006C18303C791C3D782A46303AD2B20A2A92
:10A300000F46F3D30CE001CC0028139401D51021A3
:10A310000B43C1174840441A781E057800E000241A
:10A3200000202E2D08D13D782A2D07D17D78BF1C25
:10A33000139901C9139113E00E9018E07F1C294670
:10A340003039C9B209290FD80A2141436818303879
:10A35000791C3D782A46303AD2B20A2A0F46F3D306
:10A3600000280E9001D502E00E900C980343184689
:10A37000E1172A46683AD301D2B252089A18D2B2EB
:10A38000092A2BD8920002A39A5803469746C04642
:10A39000B9A30008C3A30008CDA30008EDA30008DB
:10A3A000EDA30008EDA30008C7A30008EDA3000873
:10A3B000EDA30008C7A300083D78682D10D1082040
:10A3C00008E0022003433D787F1C0FE03D786C2DB0
:10A3D00009D1022003437D78BF1C07E0034605E056
:10A3E0007F1C042201E07F1C012213438C43462D75
:10A3F0000B941BDD2946633915292BD8139CC046C5
:10A400007944097949008F44460B421CC30A0B0A60
:10A410000A0A0A5966730A0A810A830A0A2E0FE792
:10A42000049803430021099119467AE0442D1598B8
:10A43000139C08DD452D28D0462D00D000E7079855
:10A440000343029824E0252D00D080E2252101F06D
:10A45000E6F8F5E6472D139C00D197E0582D00D083
:10A46000EEE607980343CE4A782D00D12032190634
:10A47000C81709900C98034201D0CA4803401946F6
:10A480000498099B134009934BE0079803430398F2
:10A490000343059A7EE0264624780B98421E159DBC
:10A4A000284619461292149301F00BF928462146CA
:10A4B00034460F9E01F0B3F8241DDFE0180700D5E5
:10A4C00049E29807159801682068016000D446E2C7
:10A4D0000021416043E20C980342194601D0B14883
:10A4E00001401A06D217302010400990049818E055
:10A4F000069718060C990B43C017232101400991B8
:10A5000004CC1394002708200E90B2E101CC8DE01A
:10A510000C98034201D0A348034019460498002236
:10A52000099202220A400142069706D1002A09D167
:10A53000231D002722461C460AE0002A12D104CC23
:10A54000D01715E0E21D07239A43576814460834D4
:10A5500013684A0714D408220A4000D0DBB2002A4C
:10A560000FD1FCE0E41D07229443226860680834A0
:10A570004B0708D40B0700D5DDE013460746DDE0A6
:10A580009BB20027EBE013B21204D6E00798034316
:10A59000059A13430C98034201D00E9800E0062060
:10A5A00014931340991A4A424A410E92002800D04F
:10A5B0000E90E41D0720844303CC083CFFF788FB82
:10A5C0002546044601F024F8083513950028204656
:10A5D0000ED00021FFF7E4FA149B1A4607990A40AF
:10A5E000002813D0002A704800D070482C461BE089
:10A5F00001F005F8002846D00798149B03426C48E8
:10A6000000D06C486C490B402C460FE0002A6B4987
:10A6100000D06B49002A01D0694800E067482C4609
:10A62000401C9A0600D5084663490B400028654E39
:10A6300000D0064619465B48014014910C9803422D
:10A640001394304602D1FFF70DFD02E00E99FFF79B
:10A6500023FD05460B98441B15981499224601F0DA
:10A6600030F8002D129407D0159C3178204600F068
:10A67000D6FF761C6D1EF8D1139C0F9E1498C00651
:10A6800000D4DDE55DE10126204601F080F80546B5
:10A69000002801D0F007444012961EA9204601F080
:10A6A00094F81E980A9948430A21FFF713FC0646BE
:10A6B0001E90002D03D060201499014314910025B1
:10A6C00020462946FFF72AFA002818D1701CFFF708
:10A6D00023FD01462046FFF74BFA00281E9806D0BE
:10A6E000411C1E91801CF2E71E98401E1E90FFF731
:10A6F00013FD01462046FFF753FA0028F4D1149ABF
:10A7000016460598064012998B029E4200D128E118
:10A71000864209D11E980E99814200DC22E1042173
:10A72000C943884200DC1DE112930398024200D025
:10A7300020E10E9D06E253B21206D717002F05D472
:10A740008A060AD44A060AD5202007E000225B4286
:10A75000BA412D200990174601E02B2009901A4696
:10A760000C98014201D00F4801400B460C98014261
:10A77000139401D00E9800E0012000246E2D0E905D
:10A7800039DD6F3D092D00D994E0C0467D442D7917
:10A790006D00AF44196E8F8F8F8F368F8F6EC046CE
:10A7A00058300000FFFDFFFFC7C10008C2C100080C
:10A7B00088C4000884C40008FFFEFFFFD1C1000860
:10A7C000CCC100080FBA00081046384372D0D00838
:10A7D00079074018014607201040303018AA10555C
:10A7E000C808FF087A0780180A463A43641C002A02
:10A7F0000A46EFD15EE0582D3BD0642D01D0692D83
:10A8000058D11046384355D01946169801400D913D
:10A810000021149314463B460D9800280F4608D09B
:10A8200008460A990840032803D118A82C21C155CD
:10A830007F1C0A2200252046194612932B46FFF75B
:10A8400095FB1094044611910A222B46FFF72AFB30
:10A85000109A101A3021014318A8C155791C0920FB
:10A86000801A12988541119F0F9E149BD3D30C46DA
:10A8700020E0104638431CD007981D460342FA4892
:10A8800000D0FA48134611093A07891800240A46ED
:10A890000F211940415C18AB195511093F093B07BD
:10A8A000C91813463B43641C002B1346EFD12B46BB
:10A8B00000E00024099A511E104688410B99091B9B
:10A8C000FF2A00D9491E069F081A0E990D1BE91789
:10A8D0008D43421B3342149305D11598194600F05D
:10A8E000F0FE149B0022099E310A129204D01598A2
:10A8F00000F095FE129A149B002E3146159E04D04E
:10A90000304600F08CFE129A149B3046194600F037
:10A91000D8FE302130462A4600F0A3FF012C0ADB86
:10A92000641C18A80019801E0178304600F077FEDC
:10A93000641E012CF5D81498C006139C0F9E00D4F9
:10A940007EE420211598129A00F08BFF78E4002D08
:10A9500000D075E4EBE22068159909680170241DA8
:10A960006EE41E98119626282ED12046CC49FFF77A
:10A970008BF82FE01E980E2800DDE3E0C0430E990F
:10A980000E18102E00DB1026100600D5D9E0002E80
:10A99000354600D1D6E03046FFF7BEFB2146FFF733
:10A9A00017F83F210906FEF771FFFFF74FFABD497F
:10A9B000FFF7C0F900252946FFF7B0F8002800D1BD
:10A9C000BFE0761EE7D1BDE04042FFF7A5FB214680
:10A9D000FEF7FEFF064600252946FFF79FF80028F0
:10A9E000139C15D1304600F013FE0028304611D0DC
:10A9F0000021FFF7D5F8149B1A4607990A40002852
:10AA000000D196E0002AA84800D10DE6A7480BE641
:10AA1000099527E00995A34C2146FFF78FF81E9D65
:10AA200000280BD030462146FFF72EF80646214677
:10AA3000FFF784F86D1C0028F4D11E957F20C40513
:10AA400030462146FFF7ACF800280BD03046954938
:10AA5000FEF7BEFF06462146FFF7A2F86D1E00284E
:10AA6000F4D11E950598119981420E9801D00546A2
:10AA700000E0451E8B4C0028294600D10021119191
:10AA80004842FFF749FB019900F083FE3146FEF78B
:10AA9000FDFE06462146FFF751F8002807D01E9814
:10AAA000401C1E9030462146FEF7EEFF0646149AE3
:10AAB00011980D96002839D0119502990B468033D4
:10AAC00013408B4200D0ABE0102800DB102005467D
:10AAD000FFF722FB3146FEF77BFFFFF7A3F810904C
:10AAE00008430998119000D19AE00A220023109897
:10AAF0000E46FFF73BFA002D00D190E01A4300D03C
:10AB00008DE0119531460A2200231098FFF72EFAA6
:10AB100010900C460A220023FFF728FA1198401ED5
:10AB200011907DD01A432146EDD079E0099811901B
:10AB300076E0002A5E4900D05E49002A6DD05D486B
:10AB40006EE535461E9810386942884200DC08469A
:10AB5000FFF7E2FA019900F01CFE2146FEF796FE8F
:10AB600004461E98401CFFF7D7FA01462046FEF720
:10AB7000FFFF1E99002800D0491C14980029119548
:10AB800011D4112914D3084610381E901020401AF1
:10AB9000FFF7C2FA2146FEF71BFFFFF743F8064610
:10ABA0000C46002012E00D9400261E9634460FE05D
:10ABB00000201E902046FFF735F8254606460C4635
:10ABC000FFF76EF801462846FEF7FAFE0D9014983E
:10ABD00012998843DB49083100250A4608326D1C6A
:10ABE0000B684968F31A23468B411146F6D210953B
:10ABF000119B002B0099149A01D1D1B2C9095206B8
:10AC0000920F01D1494200E0C9431E9A891A0B9A5A
:10AC1000D21A5118491B024676E0C74800E5119543
:10AC2000119D002D0098149A01D1D0B2C0090B9942
:10AC3000491B081A411F1E9C17980242129E01D1FF
:10AC400010963FE00E91032120461091FFF762F924
:10AC5000881C042822D8C0467844007940008744E4
:10AC600007132B071300C04674C4000864C400080F
:10AC7000641E1E940D98B149FEF7AAFE0D900E9920
:10AC8000491E022010901AE0A41E1E940D98AC4993
:10AC9000FEF79EFE0D900E99891E10E000200CE03C
:10ACA0009976967E00002041C7C10008C2C1000805
:10ACB000D1C10008CCC10008012010900E99149A4F
:10ACC000E81785435006800F119500D0491E0E915C
:10ACD000F502204600F08BFD632802DD0E98401E31
:10ACE0000E9014980D9CA84314902046FEF79AFFEE
:10ACF000254606460C46FEF7D3FF01462846FEF7DA
:10AD00005FFE149A0D900E99C8170D4685430F9853
:10AD100010300242149208D1012906DB2021159837
:10AD200000F07DFC6D1EF9D1149A40201040910670
:10AD300003D400280AD0202104E0002801D02D21CE
:10AD400000E02B21159800F06AFC149AD0060AD472
:10AD5000002D08D03021159800F061FC6D1EF9D14E
:10AD600000200E9000E00E951099491E0D46C80077
:10AD7000744A111849681258B01A2046884101D205
:10AD8000302007E03020B61A8C41401CB31A23460D
:10AD90008B41F8D2C1B2159800F041FC2946002D34
:10ADA0001498E2D10146029801401291159E0BD0F1
:10ADB0001E98012808DB401E1E903021304600F00E
:10ADC0002EFC1E980028F6DC802014990840119C67
:10ADD00020430E9D4BD02E21304600F020FC102C3D
:10ADE000264600DB1026F0173446844312980028CC
:10ADF00001D1204601E01E98201AFFF78DF9014687
:10AE000011981094001B0B90012E23DB0D98FEF778
:10AE1000DFFDFEF707FF04460E46109B5B1ED800C1
:10AE2000484A111849681258A01A304688411293AE
:10AE300001D2302007E03020A41A8E41401CA31A12
:10AE400033468B41F8D2C1B2159800F0E8FB129B53
:10AE5000002BE3D10B980028159E119807D010996C
:10AE60000C1A3021304600F0DAFB641CF9D3039849
:10AE7000149901423BD00798014201D0452100E0DE
:10AE80006521159C204600F0CAFB1E98002820462C
:10AE900004D42B2100F0C3FB1E9805E02D2100F007
:10AEA000BEFB1E9840421E9064280FDB6421FFF712
:10AEB00039F801463031159E304600F0B0FB1E983F
:10AEC0006421FFF727F808461E9100E026460A2174
:10AED000FFF700F801463031304600F0A0FB1E9825
:10AEE0000A21FFF717F83031304600F098FB002DAB
:10AEF000139C0F9E01D1FFF7A3F9159C202120463A
:10AF000000F08DFB6D1EF9D1139CFFF799F9159C8C
:10AF1000E068002805D006CC083C914201D2089A8E
:10AF20004254204600F0C0FB20681FB0F0BD00F086
:10AF3000BBFB0198F9E7C046D1C1000800002041E1
:08AF40000000C842C030000807
:10AF4800084B1B6883420AD0074B1B68834206D014
:10AF5800064B1B68181A431E984140427047002050
:10AF6800FCE7C046680B0020640B00206C0B002037
:04AF780040207047BE
:0CAF7C0010B5006800F0C8F810BDC04619
:10AF880003230F480F4A036143610F4B8261C3617A
:10AF98008023DB000362002383624362C36202668C
:10AFA8000A4A426610228266094A0367C3664367F3
:10AFB8001178013AC1540133102BF9D17047C046BA
:10AFC80034080020D0B20008C0000020240B002064
:04AFD800FFB20008BC
:10AFDC00F8B54746CE46C568836804004068994674
:10AFEC005B1B80B50E00170098464019934207D999
:10AFFC00FFF73AF8ED19E560C0BCB946B046F8BDAC
:10B00C001A00FFF731F84B463100ED19ED1A2A0002
:0CB01C0060684144FFF728F8EDE7C046EB
:10B02800F8B54746CE46002380B588460700160087
:10B038009946C56884681BE0013B5B1B641BB442EE
:10B0480000D934009C4200D91C007868220041468F
:10B058004019FFF70BF82D19A144A044361BBC6812
:10B06800631B5A1E93415B421D40FD60002E06D0B3
:10B078003B699D42E0D3013B1B195B1BDEE7484659
:08B08800C0BCB946B046F8BD9A
:10B0900070B50600431C5C00E4181D4BE400E0188A
:10B0A0007400A419E4001B19DC6A1500012C06D0F9
:10B0B000022C1FD0002C10D00024200070BD9A6AF2
:10B0C0005C6AA2421FD9013A121B2C00954200D99A
:10B0D00014002200FFF782FFEFE79A6A5E6AB2422D
:10B0E0000CD9013A961BB542E7D82A00FFF776FF44
:10B0F0002C00E2E7FFF798FF0400DEE71B6AD21896
:10B10000013A961BEFE71B6AD218013A121BDCE7E3
:04B1100034080020DF
:10B11400F8B50B4B04001B780D001600002B0CD067
:10B12400EFF31087012181F31088320029002000F9
:10B13400FFF7ACFF87F31088F8BDFFF723FFEFE7B5
:04B1440034080020AB
:10B14800072904D9024B4160186000230360704747
:04B15800440B002084
:10B15C0000000000000000000000000000000000E3
:10B16C0000000000000000000000000000000000D3
:10B17C0001000000020000000300000004000000B9
:10B18C000600000007000000080000000900000095
:10B19C0000000000000000000000000000000000A3
:10B1AC000100000002000000030000000400000089
:10B1BC000000000004000000020000000800000075
:10B1CC00004B0000650001000100740EF00A420EF5
:10B1DC00100E540B800CC409280AF401C201320071
:10B1EC0046006AFF9CFF5802100EFA000000000097
:10B1FC000000000000000000000000000000000043
:10B20C00DB090020DC090020DD090020DE0900201C
:0CB21C0052BD000848B2000828B200082B
:10B228002DA0000833B800083FB8000849A000085E
:10B238004BB8000857B8000823B80008F7B700084B
:10B2480054BD0008A2C10008A2C10008A2C100089C
:10B25800A2C10008A2C10008A2C10008A2C100083A
:10B26800A2C10008A2C10008FFFFFFFFFFFFFFFF08
:10B27800FFFFFFFFFFFF000056BD000854C1000894
:10B28800A2B9000871C10008F9B90008A3C10008F3
:08B29800ACC1000800BA000877
:10B2A000000020410000C84200401C4620BCBE4CAB
:08B2B000CA1B0E5AAEC59D74C5
:10B2B80003480449091A08B5FFF742FF0CBC1847B0
:08B2C800100C00201010002002
:09B2D0005465726D696E616C0039
:10B2D900455845433A20466163746F727920526537
:07B2E90073746F72650A0027
:10B2F0000000000000005454522052454747455377
:01B30000004C
:0FB30100455845433A20524553544152540A008F
:02B31000FEE756
:02B31200FEE754
:02B31400FEE752
:02B31600FEE750
:02B31800FEE74E
:02B31A00FEE74C
:02B31C00FEE74A
:02B31E00FEE748
:02B32000FEE746
:02B32200FEE744
:02B32400FEE742
:02B32600FEE740
:02B32800FEE73E
:02B32A00FEE73C
:02B32C00FEE73A
:02B32E00FEE738
:02B33000FEE736
:02B33200FEE734
:02B33400FEE732
:02B33600FEE730
:02B33800FEE72E
:02B33A00FEE72C
:02B33C00FEE72A
:02B33E00FEE728
:02B34000FEE726
:02B34200FEE724
:02B34400FEE722
:02B34600FEE720
:02B3480070474C
:10B34A0030B584214158212918D102465632938AB0
:10B35A00002B13D0016802E05B1E1C040ED0148877
:10B36A00002C0CD0CC692406F6D5046D25788D62A4
:10B37A00641C04651488641E1480EDE730BD012046
:10B38A00C0058A6882438A600868402202430A60CC
:02B39A0030BDC4
:10B39C0010B5882141582229016810D102465E322D
:10B3AC005388496A1940836D19701188491E1180A0
:10B3BC00816D491C81651188002905D010BD8869F3
:10B3CC00082202438A6110BD0246883209214B01D2
:10B3DC0001680C689C430C608B680124A3438B6050
:10B3EC002023136000220267C36E012B03D10B686C
:0AB3FC001024A3430B60C26610BDCD
:10B4060010B588214158222901680FD102465E32C3
:10B4160053884C6A1C40836D1C801488641E1480FB
:10B426009B1C83651288002A05D010BD88690822F6
:10B4360002438A6110BD0246883209235B010C680B
:10B446009C430C608B680124A3438B60202313600C
:10B4560000220267C36E012B03D10B681024A3439D
:06B466000B60C26610BD80
:02B46C00FEE7F9
:02B46E00FEE7F7
:02B47000704723
:02B47200704721
:10B4740008D1002806D1F54204D801D3002A01D10D
:10B484006D0D09D10020C143090DC904F0BDF9D1E6
:10B494001242F7D1640DF5D00020C1434905490893
:10B4A400A6E000206146F0BDF0B50127FF070E00BD
:10B4B4005E403E40B446BE0A4C18DD18F442D7D272
:10B4C400F542E4D2640DECD06D0DEAD06419C902E2
:10B4D4003943460DC0023143DB023B43DB0A10B45F
:10B4E4008E4685B297B26F43140C6C433E0CA4197C
:10B4F400260C2404BFB227439CB26C43A419190C34
:10B504006943250CA4B249190D04090C6419000CF3
:10B5140095B245433E0C76193743BFB2360C150C31
:10B524004543AD19A6B2240CAD192E0437432E0C95
:10B5340036199DB24543AD19ACB22E0C89191D0CB8
:10B5440045436D182E04290C3443704680B295B2DD
:10B5540045433E0C76193743BFB2360C150C4543B0
:10B56400AD19A6B2AD19240C2E0437432E0C36198E
:10B574009DB24543AD19ACB22E0C89191D0C45433F
:10B584006D182E043443290C75462D0C90B2684373
:10B594003E0C80190604BFB23E43070CA0B23F180C
:10B5A400120C6A43D019020C80B2240CA4189AB26B
:10B5B4006A43121914042043120C89181B0C6B43A0
:10B5C400C91810BC01273D05294203D1B6194041D1
:10B5D4004941013CFF077D0D013D641B0BDB6D0000
:10B5E400AC4209DA240500254208BE4168416141A4
:0AB5F40066463143F0BD54E74EE710
:10B5FE00FF2109064000884201D800207047012033
:02B60E00704783
:0EB61000012109064000411848424841704798
:10B61E0030B581B0044668460170206900280FD00D
:10B62E000CCC083C9A4233D26269531C636181543C
:10B63E00A069616981422BD1204600F02EF827E0E7
:10B64E00E068002809D00CCC083C9A4220D2551C48
:10B65E009D4200D1002181541AE0A068002808D034
:10B66E000CCC083C9A4213D2551C9D420DD0C9B247
:10B67E000CE0236A002B0BD003CC083C884207D287
:10B68E00694601222046984702E00021920081502F
:0AB69E002068401C206001B030BDA0
:10B6A80010B54269002A07D00446036A002B01D06E
:0AB6B800216998470020606110BD71
:10B6C20080B5CB0606D4890501D5302100E02021C2
:06B6D20000F0C6F880BD87
:10B6D80070B514460D460646FEF798FC01463046FE
:0AB6E8002A462346FEF738FD70BD28
:08B6F200F7F73FFDF7F733FD08
:10B6FA00806A816D40220A438265C16D04220A4331
:04B70A00C26570475D
:10B70E0010B58421415821290DD1014656310A88A0
:10B71E00002A09D00268036D1C7894625A1C0265D7
:10B72E000888401E088010BD006801688022914381
:0CB73E000160016840220A43026010BD57
:08B74A0080B5FDF762FF80BD30
:08B7520080B5FDF75EFF80BD2C
:10B75A00F0B581B01E4615460C4607461846FFF757
:10B76A00EEFB0146002000290AD46543A54207D30F
:10B77A00304639462A46FFF7FCFB2146FEF7CDFB49
:04B78A0001B0F0BD5D
:04B78E00C00F704731
:10B7920010B5FD22D343C20DD2B21446FF3C9C42E7
:10B7A20008D351184A1EFD2A05D8FF22D20590431C
:10B7B200C905084310BD0122D20710400129F9DB57
:08B7C200FF21C905401810BD6C
:10B7CA00C20DD2B2FF2A01D0002A02D100220A6099
:10B7DA0070477E3A0A60FF21C90588433F2109065E
:04B7EA00401870474C
:08B7EE00C1174840401A7047E2
:10B7F60010B5002A0DD00446097848B200280AD4AC
:10B80600002C00D02160002119605960411E88413A
:0CB8160010BD002010BD0120C04310BD7B
:10B82200024601207F2901D9C04370471170704739
:0CB83200014661391A2900D22038704705
:0CB83E00014641391A2900D22030704721
:0CB84A00014661391A2900D220387047ED
:0CB85600014641391A2900D22030704709
:10B8620070B5012A09DB0C460546561C28462146BE
:0CB87200FFF7D4FE761E012EF8D870BD42
:10B87E0010B50C46436A01212046FFF767FF10BD45
:10B88E00010002000400060008000A000C0010006F
:08B89E002000400080000001C1
:10B8A6006E6F7420616C6C6F7765642C20706172AA
:0FB8B600616D746572206C6F636B6564210A00AD
:10B8C50048414C5F434F4D50315F53746172742052
:07B8D5004552524F520A00D8
:10B8DC0048414C5F434F4D50325F5374617274203A
:07B8EC004552524F520A00C1
:10B8F300434F4E564552544552204552524F523AA9
:10B9030020434F4E5645525445525F53544152546F
:0BB913005550204552524F52210A00AF
:10B91E00434F4E564552544552204552524F523A7D
:10B92E0020434F4E5645525445525F4552524F5248
:10B93E005F4F55545055545F564F4C545F544F4FB4
:07B94E005F484947480A0069
:10B9550042617474657269652063686172676564C4
:10B9650021204379636C65636F756E7465722B2B4B
:03B97500210A00A4
:10B9780048414C5F4144435F53746172745F444D66
:07B98800413A204F4B0A0079
:10B98F002D3E4D65737361676520746F2073686F0B
:03B99F00727400BF
:10B9A2004A616E756172790046656272756172797B
:10B9B200004D6172636800417072696C004D61797B
:10B9C200004A756E65004A756C790041756775733A
:10B9D200740053657074656D626572004F63746FB5
:10B9E200626572004E6F76656D62657200446563D2
:07B9F200656D626572000043
:07B9F900414D00504D00001C
:0FBA000025612025622025652025542025590029
:07BA0F00286E756C6C290024
:10BA1600443A5C70726F6A656B74655C6563735FEC
:10BA2600677265656E506F7765725061636B5C65B2
:10BA360063735F63656C6C4D6F6E5C6669726D7780
:10BA46006172655C447269766572735C53544D33FA
:10BA560032473078785F48414C5F44726976657248
:10BA66005C5372635C73746D3332673078785F68E9
:0ABA7600616C5F636F6D702E63005A
:10BA8000443A5C70726F6A656B74655C6563735F82
:10BA9000677265656E506F7765725061636B5C6548
:10BAA00063735F63656C6C4D6F6E5C6669726D7716
:10BAB0006172655C447269766572735C53544D3390
:10BAC00032473078785F48414C5F447269766572DE
:10BAD0005C5372635C73746D3332673078785F687F
:0EBAE000616C5F666C6173685F65782E630051
:10BAEE00443A5C70726F6A656B74655C6563735F14
:10BAFE00677265656E506F7765725061636B5C65DA
:10BB0E0063735F63656C6C4D6F6E5C6669726D77A7
:10BB1E006172655C447269766572735C53544D3321
:10BB2E0032473078785F48414C5F4472697665726F
:10BB3E005C5372635C73746D3332673078785F6810
:0ABB4E00616C5F6770696F2E630081
:10BB5800443A5C70726F6A656B74655C6563735FA9
:10BB6800677265656E506F7765725061636B5C656F
:10BB780063735F63656C6C4D6F6E5C6669726D773D
:10BB88006172655C447269766572735C53544D33B7
:10BB980032473078785F48414C5F44726976657205
:10BBA8005C5372635C73746D3332673078785F68A6
:0ABBB800616C5F756172742E63000A
:10BBC200666163746F726520726573746F7265204B
:0ABBD2002850696E292E2E2E0A005D
:10BBDC004558453A2053746F726520706172616DDF
:06BBEC00657465720A0099
:10BBF200455845433A204170706C79204D4220509F
:0ABC02006172616D657465720A00DD
:10BC0C00455845433A20526573657420436F756EF1
:06BC1C00746572730A005A
:10BC220048414C5F4441435F5374617274204F4BEF
:02BC32000A0006
:10BC340042414C414E4345525F496E6974204F4B1B
:02BC44000A00F4
:10BC4600434F4E564552544552204552524F523A52
:10BC560020434F4E5645525445525F4552524F521D
:10BC66005F4F55545055545F564F4C545F544F4F89
:06BC76005F4C4F570A006D
:10BC7C00426174746572696520646973636861728A
:06BC8C00676564210A0057
:10BC92004D696E75746520496E74657276616C6C5F
:0ABCA20020636865636B73210A00DC
:10BCAC004E6577204D696E20566F6C746167652008
:0ABCBC0025642053617665640A00D8
:10BCC6004E6577204D617820566F6C7461676520EC
:0ABCD60025642053617665640A00BE
:10BCE000466972737420737461727420646574653C
:06BCF000637465640A00A4
:10BCF600454550524F4D2046554C4C2052455354C5
:06BD06004F5245210A0026
:10BD0C00454550524F4D2053544F524520434F4EB2
:06BD1C00464947210A0020
:10BD22004572726F72207768696C652073617669FB
:10BD32006E67206461746120746F20666C61736841
:02BD42000A00F5
:0EBD440075617274206572726F72200A0D00B4
:02BD52004300AC
:02BD54002E00BF
:10BD560053756E646179004D6F6E64617900547538
:10BD66006573646179005765646E65736461790013
:10BD7600546875727364617900467269646179000A
:0ABD86005361747572646179000066
:10BD9000443A5C70726F6A656B74655C6563735F6F
:10BDA000677265656E506F7765725061636B5C6535
:10BDB00063735F63656C6C4D6F6E5C6669726D7703
:10BDC0006172655C447269766572735C53544D337D
:10BDD00032473078785F48414C5F447269766572CB
:10BDE0005C5372635C73746D3332673078785F686C
:09BDF000616C5F6164632E630065
:10BDF900443A5C70726F6A656B74655C6563735F06
:10BE0900677265656E506F7765725061636B5C65CB
:10BE190063735F63656C6C4D6F6E5C6669726D7799
:10BE29006172655C447269766572735C53544D3313
:10BE390032473078785F48414C5F44726976657261
:10BE49005C5372635C73746D3332673078785F6802
:09BE5900616C5F6461632E6300FB
:10BE6200443A5C70726F6A656B74655C6563735F9C
:10BE7200677265656E506F7765725061636B5C6562
:10BE820063735F63656C6C4D6F6E5C6669726D7730
:10BE92006172655C447269766572735C53544D33AA
:10BEA20032473078785F48414C5F447269766572F8
:10BEB2005C5372635C73746D3332673078785F6899
:09BEC200616C5F646D612E630088
:10BECB00443A5C70726F6A656B74655C6563735F33
:10BEDB00677265656E506F7765725061636B5C65F9
:10BEEB0063735F63656C6C4D6F6E5C6669726D77C7
:10BEFB006172655C447269766572735C53544D3341
:10BF0B0032473078785F48414C5F4472697665728E
:10BF1B005C5372635C73746D3332673078785F682F
:09BF2B00616C5F74696D2E630006
:10BF3400443A5C70726F6A656B74655C6563735FC9
:10BF4400677265656E506F7765725061636B5C658F
:10BF540063735F63656C6C4D6F6E5C6669726D775D
:10BF64006172655C447269766572735C53544D33D7
:10BF740032473078785F48414C5F44726976657225
:10BF84005C5372635C73746D3332673078785F68C6
:0DBF9400616C5F756172745F65782E6300EB
:10BFA10066756C6C20726573746F72652E2E2E0A25
:01BFB100008F
:10BFB200455845433A2053746F7265207769746817
:05BFC20020736E0A006F
:10BFC700455845433A2053617665206C6F636B2073
:05BFD7006B65790A0012
:10BFDC00554E4B4E4F574E20434F4D4D414E440AFC
:01BFEC000054
:10BFED0057726F6E6720706172616D6574657273E3
:10BFFD002076616C75653A2066696C652025732025
:0DC00D006F6E206C696E652025640D0A00C1
:10C01A0048414C5F4441435F53657456616C756592
:05C02A00204F4B0A004D
:10C02F0048414C5F4441435F5374617274204552E1
:05C03F00524F520A00FF
:10C0440044432044432057616E646C6572206E6FD4
:10C05400742072756E6E696E672C207374617274CD
:09C0640020696D70756C730A000F
:10C06D0070726576696F757320636F6E6669672090
:09C07D0070726573656E740A00AF
:0DC0860057726974696E6720534E210A00DD
:10C093004572726F72207768696C652064656C65A0
:10C0A30074696E67206C6F672064617461206172CC
:0DC0B300656120696E20666C6173680A008B
:10C0C00048414C5F41444345785F43616C6962720B
:10C0D0006174696F6E5F53746172743A204F4B0ADA
:01C0E000005F
:10C0E1004572726F722048414C5F4144435F537403
:09C0F1006172745F444D410A00C4
:10C0FA002D3E4D6573736167652077697468207793
:09C10A00726F6E6720637263001E
:10C11300443A5C70726F6A656B74655C6563735FE8
:10C12300677265656E506F7765725061636B5C65AE
:10C1330063735F63656C6C4D6F6E5C6669726D777C
:10C143006172655C7372635C6D6F646275732E6399
:01C1530000EB
:10C1540053756E004D6F6E0054756500576564002D
:0DC164005468750046726900536174000054
:10C171004A616E00466562004D6172004170720055
:10C181004D6179004A756E004A756C004175670012
:10C19100536570004F6374004E6F76004465630011
:01C1A100009D
:01C1A200009C
:09C1A300256D2F25642F2579007C
:09C1AC0025483A254D3A255300BF
:0DC1B5000007032004170201085710408006
:05C1C2002D494E46006E
:05C1C7002D696E660009
:05C1CC002B494E460066
:05C1D1002B696E660001
:02C1D600FFFF69
:04C1D80085310008A5
:10C1DC00443A5C70726F6A656B74655C6563735F1F
:10C1EC00677265656E506F7765725061636B5C65E5
:10C1FC0063735F63656C6C4D6F6E5C6669726D77B3
:10C20C006172655C447269766572735C53544D332C
:10C21C0032473078785F48414C5F4472697665727A
:10C22C005C5372635C73746D3332673078785F681B
:0CC23C00616C5F6164635F65782E6300D5
:10C24800443A5C70726F6A656B74655C6563735FB2
:10C25800677265656E506F7765725061636B5C6578
:10C2680063735F63656C6C4D6F6E5C6669726D7746
:10C278006172655C447269766572735C53544D33C0
:10C2880032473078785F48414C5F4472697665720E
:10C298005C5372635C73746D3332673078785F68AF
:0CC2A800616C5F74696D5F65782E630047
:08C2B400010101030701000074
:08C2BC0008040204080101015D
:10C2C4007265616420636F6E6669672E2E2E0A00A4
:10C2D400455845433A205265736574204D696E2074
:10C2E400616E64204D61782056616C7565730A0037
:10C2F40048414C5F434F4D50315F53746172742019
:04C304004F4B0A0091
:10C3080048414C5F434F4D50325F53746172742003
:04C318004F4B0A007D
:10C31C004E6577204D696E2054656D702E20256416
:08C32C002053617665640A00EC
:10C334004E6577204D61782054656D702E202564FC
:08C344002053617665640A00D4
:10C34C00486F757220496E74657276616C6C2063EF
:08C35C006865636B73210A00A0
:10C36400454550524F4D2053544F5245204C4F4752
:08C374002044415441210A005C
:10C37C0048414C5F41444345785F43616C6962724C
:10C38C006174696F6E5F53746172743A20455252D6
:04C39C004F520A00F2
:10C3A0004572726F722C2072656164206F6E6C79B9
:0CC3B000205265676973746572210A00F1
:10C3BC0050726F7465637465642052656769737439
:10C3CC0065722C207772697465206E6F7420616CB5
:08C3DC006C6F776564210A0013
:10C3E40020202020202020202068282828282020E1
:10C3F4002020202020202020202020202020202039
:10C4040048101010101010101010101010101010F0
:10C414008484848484848484848410101010101090
:10C4240010818181818181010101010101010101E9
:10C43400010101010101010101010110101010109D
:10C4440010828282828282020202020202020202BA
:10C454000202020202020202020202101010102062
:10C464003031323334353637383941424344454626
:10C474003031323334353637383961626364656656
:04C484004E414E00D7
:04C488006E616E0073
:10C48C0000B506480649884205D00268043003B45A
:10C49C00904703BCF7E708BC18470000D8C1000858
:04C4AC00DCC10008E7
:10C4B00019C5000800000020480B00002BC500082B
:10C4C000480B0020D4C40008B9B200088DC400088D
:04C4D0006B310008C4
:10C4D400181CB200081CB200081CB200081CB200F0
:10C4E400081CB200080024F4000AFE000F340B00FC
:10C4F40020380B00203C0B002000000202FD00FD50
:10C5040002010101FB00E70204010000010298009E
:04C5140080000000A3
:10C51800206861680834002200E042540139FCD5E3
:02C5280070475A
:10C52A002068616808340A780131802A11D009D359
:10C53A000B7801315242FF32013203700130013A65
:10C54A00FBD5F0E70B78037001300131013AF9D5D8
:04C55A00E9E7704756
:10C55E00FFFFFFFFFFFFFFFFFFFFFFFFFFFFFFFFDD
:10C56E00FFFFFFFFFFFFFFFFFFFFFFFFFFFFFFFFCD
:10C57E00FFFFFFFFFFFFFFFFFFFFFFFFFFFFFFFFBD
:10C58E00FFFFFFFFFFFFFFFFFFFFFFFFFFFFFFFFAD
:02FFFE00FFFF03
:020000040801F1
:10000000FFFFFFFFFFFFFFFFFFFFFFFFFFFFFFFF00
:10001000FFFFFFFFFFFFFFFFFFFFFFFFFFFFFFFFF0
:10002000FFFFFFFFFFFFFFFFFFFFFFFFFFFFFFFFE0
:10003000FFFFFFFFFFFFFFFFFFFFFFFFFFFFFFFFD0
:04EFFC00187F071D56
:040000050800B6F346
:00000001FF
